:100000002BC3000048C3000046C3000044C30000E7
:1000100042C3000040C300003EC300003CC30000D8
:100020003AC3000038C3000036C3000034C30000E8
:100030000C94CD3E30C300002EC300002CC3000042
:100040002AC3000028C300000C94B93E24C300005A
:1000500022C3000020C300001EC300001CC3000018
:100060001AC3000018C3000016C3000014C3000028
:1000700012C3000010C300000EC300000CC3000038
:100080000AC3000008C3000006C30000510F980F08
:10009000C80FF80F50106B109B10D2103B110211BB
:1000A000760F7B0FCD10F710FC10890F8E0F930F7A
:1000B00088139313951397139A139D13B713B913BA
:1000C000C613D213D516DA16E816ED16F216F71681
:1000D000FC160117951B981B9B1B9E1BA11BA41BA9
:1000E000A71BAA1B78259D25B125C425C725D82582
:1000F000E92507268E259125FA25FD25002694253C
:1001000097259A25042B092B0E2B132B182B1D2B0F
:10011000222B272B2C2B2F2BE32C4E2D722EDB2E5C
:10012000FA2F26310C32013330347F34E2342C354F
:1001300033358735DC35DF35E235E535E835EB3508
:10014000EE35F1358D38A338B938D038E638FC387B
:10015000123928397C397F398239853988398B3988
:100160008E399139CB39E039F539083A1B3A293AB9
:100170003C3A4F3A623A773A8C3AA13AC03AD93A85
:10018000000000000000000004040404000400005B
:100190000A0A0A00000000000A0A1F0A1F0A0A00D1
:1001A000040F140E051E040018190204081303009E
:1001B0000C12140814120D000C04080000000000BA
:1001C00002040808080402000804020202040800ED
:1001D0000004150E150400000004041F04040000B0
:1001E000000000000C0408000000001F00000000D8
:1001F00000000000000C0C000001020408100000C8
:100200000E11131519110E00040C040404040E0041
:100210000E11010204081F001F02040201110E004A
:1002200002060A121F0202001F101E0101110E0019
:100230000608101E11110E001F0102040808080014
:100240000E11110E11110E000E11110F01020C00F2
:100250000001020408100000000C0C000C0408004F
:10026000020408100804020000001F001F00000024
:1002700008040201020408000E1101020400040037
:100280000E11010D15150E000E1111111F11110087
:100290001E11111E11111E000E11101010110E0052
:1002A0001C12111111121C001F10101E10101F0023
:1002B0001F10101E101010000E11101711110E003B
:1002C0001111111F111111000E04040404040E0079
:1002D0000702020202120C0011121418141211006B
:1002E0001010101010101F00111B15151111110006
:1002F00011111915131111000E11111111110E0008
:100300001E11111E101010000E11111115120D00EA
:100310001E11111E141211000F10100E01011E00EB
:100320001F040404040404001111111111110E0022
:1003300011111111110A04001111111115150E00DE
:1003400011110A040A1111001111110A0404040008
:100350001F01020408101F000E08080808080E00FC
:10036000110A1F041F0404000E02020202020E0002
:10037000040A1100000000000000000000001F003F
:10038000080400000000000000000E010F110F0023
:1003900010101E1111111E0000000E1010110E0081
:1003A00001010D1311110F0000000E111F100E009E
:1003B0000609081C08080800000F11110F010E00A3
:1003C000101016191111110004000C0404040E0081
:1003D0000200060202120C0010101214181412006F
:1003E0001808080808081C0000001A15151111004B
:1003F000000016191111110000000E1111110E004C
:1004000000001E111E10100000000F110F0101004E
:10041000000016191010100000000E100E011E0032
:1004200008081C08080906000000111111130D002E
:1004300000001111110A04000000111111150A0029
:100440000000110A040A1100000011110F010E0032
:1004500000001F0204081F00384444447C44440048
:100460007C404078444478007844447844447800A0
:100470007C404040404040000C14242424243C4450
:100480007C40407840407C005454543854545400CC
:10049000384404180444380044444C546444440030
:1004A00054444C5464444400444850605048440010
:1004B0001C24242424246400446C545444444400E4
:1004C0004444447C44444400384444444444380054
:1004D0007C444444444444007844447840404000D0
:1004E00038444040404438007C1010101010100078
:1004F0004444443C044438003854545438101000E8
:1005000044442810284444004444444444447E0263
:10051000444444443C0404005454545454547C0013
:100520005454545454547E026020203824243800FB
:100530004444446454546400404040784444780047
:100540003844041C0444380048545474545448003B
:100550003C44443C14244400000038043C443C0027
:1005600000007840784478000000784C784C78009F
:1005700000007840404040000000182828287C44B3
:10058000000038447C403C0000005454385454006F
:1005900000007804380478000000444C546444009F
:1005A0000010444C54644400000044487048440027
:1005B00000001C24444444000000446C5454440093
:1005C0000000484878484800000038444444380057
:1005D00000007848484848000000704870404000DB
:1005E000000038404040380000007C10101010001F
:1005F0000000484838087000000038545438100093
:1006000000004428102844000000484848487C0462
:1006100000004848380808000000545454547C0036
:100620000000545454547E02000060203C223C00E0
:1006300000004242724A7200000040407844780054
:10064000000070087808700000004C5272524C0094
:1006500000003C443C44440011241FBECFEFD0E1D5
:10066000DEBFCDBF16E0A0E0B1E0EAEEFEE800E0BC
:100670000BBF02C007900D92A633B107D9F726E051
:10068000A6E3B6E001C01D92A43FB207E1F70E94C5
:100690002B3F0C947347B4CCA89521E0209382069D
:1006A0002091E1063091E2062937310578F1209159
:1006B0009A0630919B062635310540F5BC012B5F2B
:1006C0003F4F30939B0620939A061092E2061092B9
:1006D000E10690913706892F90E0880F991F80508E
:1006E00090400E947047809137068F5F8093370655
:1006F000A49A80E185BBA8952FEF81EE94E021506C
:1007000080409040E1F700C0000015BA0895409184
:100710003606E42FF0E0EE0FFF1FE050FF4F608140
:10072000718121E0240F209336066817790720F5A0
:10073000E22FF0E0EE0FFF1FE050FF4F608171816C
:100740008617970760F455E0259F900111242250E9
:10075000310930939B0620939A06409336062091E8
:10076000AB063091AC068217930730F484E190E039
:1007700090939B0680939A068091970690E0209133
:100780009A0630919B068217930720F490939B065C
:1007900080939A060895CF93DF9300D000D0CDB711
:1007A000DEB78091630080FD6BC01C821B821A82C1
:1007B0001982BE016F5F7F4FCE0103960E94954262
:1007C0008B819C818531954098F08B819C8188320A
:1007D0009A4070F489819A818431954048F48091DF
:1007E000E8069091E90601969093E9068093E80661
:1007F0008B819C818937954098F08B819C818932CF
:100800009A4070F089819A818431954048F48091B2
:10081000E8069091E90601979093E9068093E8062F
:100820008B819C818531954098F08B819C818832A9
:100830009A4070F489819A81853C994048F0809172
:100840009A0690919B06019690939B0680939A0638
:100850008B819C818937954098F08B819C8189326E
:100860009A4070F089819A81853C994048F0809146
:100870009A0690919B06019790939B0680939A0607
:100880000F900F900F900F90DF91CF910895EF92FE
:10089000FF920F931F93CF93DF9300D000D0CDB77B
:1008A000DEB78091340190913501A0913601B0916D
:1008B000370189839A83AB83BC8303E02FEF3FEF3B
:1008C0004CED50E068E470E080E090E0EED72FEF70
:1008D0003FEF4CED50E06FE770E080E090E0E5D74F
:1008E0002FEF3FEF4CED50E066EB70E080E090E0E2
:1008F000DCD72FEF3FEF4CED50E06DEE70E080E085
:1009000090E0D3D72FEF3FEF45EA50E068E470E086
:1009100080E090E00E94CA0C2FEF3FEF45EA50E0E4
:1009200068E470E087E390E00E94CA0C2FEF3FEF8D
:1009300045EA50E068E470E08EE690E00E94CA0C60
:100940002FEF3FEF4EE650E068E470E085EA90E07C
:100950000E94CA0C2FEF3FEF48EA50E068E470E0D5
:100960008CED90E00E94CA0CEE24E394F12C2FE170
:1009700030E04FEF5FEF6AE570E08CE090E048D741
:1009800095E0E92EF12C2FE130E04FEF5FEF61E9C8
:1009900070E08CE090E03CD729E0E22EF12C2FE1D2
:1009A00030E04FEF5FEF68EC70E08CE090E030D724
:1009B00032E0E32EF12C2FE130E04FEF5FEF6AE5FC
:1009C00070E083E490E024D746E0E42EF12C2FE1A0
:1009D00030E04FEF5FEF61E970E083E490E018D71B
:1009E000E12CF12C2FE130E04FEF5FEF68EC70E08D
:1009F00083E490E00DD753E0E52EF12C2FE130E0B9
:100A00004FEF5FEF6AE570E08AE790E001D767E0BB
:100A1000E62EF12C2FE130E04FEF5FEF61E970E05F
:100A20008AE790E0F5D674E0E72EF12C2FE130E074
:100A30004FEF5FEF6AE570E081EB90E0E9D6E8E028
:100A4000EE2EF12C2FE130E04FEF5FEF61E970E027
:100A500081EB90E0DDD6E12CF12C2FE130E04FEF7F
:100A60005FEF68EC70E089E890E0D2D62FE130E0EB
:100A70004FEF5FEF68EC70E083EA90E0C9D6F3E0F7
:100A8000EF2E0FEF1FEF2CE330E04AE550E068E473
:100A900070E081EE90E0F3D7CE0101967C0102E098
:100AA0002FE130E040E058EF64E670E085EF90E041
:100AB00069D6A3E0EA2E0FEF1FEF20E530E04AE50C
:100AC00050E066E970E081EE90E0D9D700EE17E0E3
:100AD0002CED30E04EE051E06EEB70E085EF90E001
:100AE0000E94BC0D20EA30E04CE251E06CED70E079
:100AF0008EE091E00E94BC0D2CED30E04FE051E023
:100B00006EEB70E086EF90E00E94BC0D20EA30E0D2
:100B10004BE251E06CED70E08DE091E00E94BC0D85
:100B20002CED30E040E151E06EEB70E087EF90E0BB
:100B30000E94BC0D20EA30E04AE251E06CED70E02A
:100B40008CE091E00E94BC0D2CED30E041E151E0E1
:100B50006EEB70E088EF90E00E94BC0D20EA30E080
:100B60004AE251E06CED70E08BE091E00E94BC0D38
:100B7000B2E0EB2E0FEF1FEF2CE330E040EA50E045
:100B800063E070E080E590E07AD70F900F900F90CF
:100B90000F90DF91CF911F910F91FF90EF900895EB
:100BA000EF920F931F9383E0E82E0FEF1FEF22E3E6
:100BB00030E040EA50E064E670E084E190E05FD726
:100BC00020E530E04AE550E066E970E081EE90E033
:100BD00056D700EE17E02CED30E04EE051E06EEB22
:100BE00070E085EF90E0C8D720EA30E04CE251E0B9
:100BF0006CED70E08EE091E0BFD72CED30E04FE07F
:100C000051E06EEB70E086EF90E0B6D720EA30E07E
:100C10004BE251E06CED70E08DE091E0ADD72CED52
:100C200030E040E151E06EEB70E087EF90E0A4D758
:100C300020EA30E04AE251E06CED70E08CE091E0B7
:100C40009BD72CED30E041E151E06EEB70E088EF96
:100C500090E092D720EA30E04AE251E06CED70E09B
:100C60008BE091E089D71F910F91EF900895EF925B
:100C7000FF920F931F93CF93DF9300D000D0CDB797
:100C8000DEB77C018091630080FD22C11C821B8243
:100C90001A821982BE016F5F7F4FCE0103960E94B8
:100CA00095420FE110E02DE230E042E550E06AE0CD
:100CB00070E08BE990E071D48B819C81893B9B40F3
:100CC00068F089819A81883D9E4040F489819A81AB
:100CD00089349D4018F089E0809325018B819C81A7
:100CE0008F32994090F08B819C81803F9A4068F4CC
:100CF00089819A81883D9E4040F489819A81893416
:100D00009D4018F085E0809325018B819C81853A78
:100D1000964090F08B819C818C3F984068F489814B
:100D20009A81883D9E4040F489819A8189349D4012
:100D300018F081E0809325018B819C81853A964053
:100D400090F08B819C818C3F984068F489819A81D6
:100D500088349D4040F489819A818D389A4018F0FA
:100D600082E0809325018B819C818F32994090F0A5
:100D70008B819C81803F9A4068F489819A81883474
:100D80009D4040F489819A818D389A4018F086E020
:100D9000809325018B819C81893B9B4060F08981F8
:100DA0009A8188349D4038F489819A818D389A409F
:100DB00010F0109225018B819C81893B9B4068F04B
:100DC00089819A818E3B9A4040F489819A818F3043
:100DD000964018F08AE0809325018B819C81853AAA
:100DE000964090F08B819C818C3F984068F489817B
:100DF0009A818C389A4040F489819A81813D97404C
:100E000018F083E0809325018B819C81853A964080
:100E100090F08B819C818C3F984068F489819A8105
:100E2000803D974040F489819A818D3D954018F02E
:100E300084E0809325018B819C818F32994090F0D2
:100E40008B819C81803F9A4068F489819A818C389B
:100E50009A4040F489819A81813D974018F087E05B
:100E6000809325018B819C818F32994090F08B81FA
:100E70009C81803F9A4068F489819A81803D9740A7
:100E800040F489819A818D3D954018F088E08093E7
:100E900025018B819C818D3D954068F08B819C81E3
:100EA0008C3F984040F489819A818C3D954018F49C
:100EB0008BE0809325018B819C818F32994040F09B
:100EC00089819A818C3D954018F48CE080932501AE
:100ED000809125018A3088F490913A0691110DC0D5
:100EE0008093480690E0909339068093380682E01C
:100EF00080933A068EE080932501809125018A3007
:100F0000A9F48091480634E6839FC0011124909390
:100F100039068093380622E020933A06E816F9064F
:100F200010F08EE001C08BE08093250180912501B7
:100F30008A30C0F490913A069230A1F4809346062C
:100F40002091480690E04AE0249F800D911D1124D5
:100F5000909339068093380683E080933A068EE0BA
:100F600080932501209125012A3010F580913A06C1
:100F70008330F1F42093470630914806809146066D
:100F80004AE0849FC001112444E6349F800D911DE6
:100F90001124820F911D909339068093380621E029
:100FA00020933A06E816F90668F48BE08093250151
:100FB000809125018B3049F4109239061092380641
:100FC00010923A068EE080932501809125018C30A5
:100FD00019F483E2809325010F900F900F900F90EA
:100FE000DF91CF911F910F91FF90EF900895EF92B5
:100FF000FF920F93E0903806F09039062AE0E2164F
:10100000F10450F403E02FE130E04FEF5FEF66E1D1
:1010100070E088EC90E0FCD3E0903806F090390660
:10102000C7010A978A35910550F403E02FE130E0BB
:101030004FEF5FEF66E170E084EB90E0E9D3E09082
:101040003806F0903906C7018456910984389340D8
:1010500050F403E02FE130E04FEF5FEF66E170E026
:101060008BE990E0D5D30F91FF90EF9008950F9307
:101070001F93CF93DF93EC018B01809125018E317B
:1010800018F48FE190E0FED31093390600933806F0
:10109000809125018E3128F4FADBCE01E8DDA7DF4F
:1010A000F7CF8FE190E0EED380913806909139062A
:1010B000DF91CF911F910F9108958EE080932501CC
:1010C0000895EF92FF920F931F93CF93DF93CDB7C5
:1010D000DEB728970FB6F894DEBF0FBECDBF809164
:1010E000630080FD50C018861F821E821D82BE01D3
:1010F0006B5F7F4FCE0107960E9495420FE110E093
:101100002EE230E044E650E062E370E082E390E0FB
:1011100044D28F819885853A964090F08F8198854A
:101120008C389A4068F48D819E8184379E4040F4CB
:101130008D819E81813F9A4018F081E08093250146
:101140008F819885853A964088F08F8198858C3874
:101150009A4060F48D819E818C389A4038F48D815C
:101160009E818939984010F0109225018F819885D1
:101170008F32994040F08D819E818C3D954018F4CE
:101180008CE08093250180912501813011F48093BA
:10119000240180912401813061F580913801909182
:1011A0003901A0913A0189839A83AB83CE010196DC
:1011B0007C0104E02FE130E040EE57E062E370E0B4
:1011C00086E490E0DFD200EE17E02EE230E04DE45E
:1011D00050E067E670E087E190E0DFD10FE110E0DA
:1011E0002EE230E04DE450E067E670E086E690E005
:1011F000D4D180912501811102C0109224018091E7
:10120000240181112FC080913B0190913C01A0915C
:101210003D01B0913E0189839A83AB83BC8300E09A
:1012200018EF2EE230E04DE450E067E670E086E62D
:1012300090E0B3D10FE110E02EE230E04DE450E059
:1012400067E670E087E190E0A8D1CE0101967C01CD
:1012500004E02FE130E040E058EF62E370E087E324
:1012600090E090D2809125018C3019F483E2809334
:10127000250128960FB6F894DEBF0FBECDBFDF91D3
:10128000CF911F910F91FF90EF900895CF93C82FAA
:10129000809125018E3118F48FE190E0F3D2C09354
:1012A0002401809125018E3120F4A89579DC09DF95
:1012B000F8CF8FE190E0E6D280912401CF9108959C
:1012C000E2E6F0E090819E7F90839081946090832D
:1012D0009081977F9083A8988BBB8DE08A95F1F7DA
:1012E0000000A89A8081886080830895E2E6F0E09B
:1012F0009081916090839081946090839081977F9A
:101300009083A8988BBB8DE08A95F1F70000A89A8E
:101310008081886080830895CF93C82F892FE6DF6E
:101320008C2FCF91E3CFE2E6F0E020812160208393
:101330002081246020832081277F2083A8988BBB75
:1013400092BB8DE08A95F1F70000A89A80818860B1
:1013500080830895CF93C82F86E3B2DFC13049F070
:1013600030F0C23041F0C33059F488EE07C088E451
:1013700003C088E203C088E8B9DF04C0B7DF0BC050
:10138000CD7F49F48FEE90E090933E0680933D062A
:101390008FE391E008C08FE391E090933E06809345
:1013A0003D068FEE90E090933C0680933B06CF91F4
:1013B0000895CF93C82F8FEF8ABB81BB80936100C4
:1013C00081E084BBE2E6F0E080818260808381E09E
:1013D00077DF2FEF89E698E1215080409040E1F7D8
:1013E00000C0000080EC6CDF85E280DF81EC68DF0C
:1013F00081E17CDF85EC64DF8BE278DF8BE276DFF6
:1014000087EC5EDF86E872DF8C2FA4DF8AE358DF8B
:1014100085E06CDF81EB54DF80E068DF88E166DF28
:1014200086EB4EDF8AE062DF82E860DF87E25EDF24
:1014300081E146DF2FEF8DEE92E021508040904019
:10144000E1F700C0000089E2CF913ACF0F931F93DC
:10145000CF93DF938C01EB018AE232DFC8015CDFBE
:10146000CE01DF91CF911F910F9156CF0F931F9314
:10147000CF93DF938C01EB018BE222DFC8014CDFBD
:10148000CE01DF91CF911F910F9146CFCF93DF9384
:10149000EB01BC01DBDFBE01CE01E8DF8CE2DF91B6
:1014A000CF910ECFCF93DF93EA01F0DFCE01DF9132
:1014B000CF9139CF8F929F92AF92BF92CF92DF920E
:1014C000EF92FF920F931F93CF93DF93A895681726
:1014D000790738F48627972768277927862797275B
:1014E000A8952417350738F4422753272427352792
:1014F00042275327A895A0913D06B0913E06FC01D6
:10150000A817B90708F4FD016B01A617B70708F47F
:101510006D0180913B0690913C06EA018417950786
:1015200008F4EC0179018217930708F47C01A8956F
:1015300096012F5F3F4F2E1B3F0BD7011196AC1B1F
:10154000BD0B0E943B444B015C01B601CF017EDF25
:10155000A895B701CE018ADF8CE2B2DEA895C12C36
:10156000D12C7601C814D904EA04FB0449F0C8015F
:10157000DADEA8958FEFC81AD80AE80AF80AF2CF7F
:10158000DF91CF911F910F91FF90EF90DF90CF905F
:10159000BF90AF909F908F9008950F931F93411528
:1015A000510579F02115310561F0FA01AB01615067
:1015B0007109260F371FBC01615071096E0F7F1F23
:1015C00079DF1F910F9108952F923F924F925F9272
:1015D0006F927F928F929F92AF92BF92CF92DF9243
:1015E000EF92FF920F931F93CF93DF93CDB7DEB7A8
:1015F00067970FB6F894DEBF0FBECDBF5C01798B45
:10160000688B598748873B872A870F83F12C28E00E
:10161000029FC00111241A821982E8E0F0E0FF8BDA
:10162000EE8B47019C01285F31093B8B2A8BFC0123
:10163000E052F340FD8BEC8BC888D98889819A8170
:10164000C80ED91E8A899B89EE89FF898E1B9F0B44
:101650009C0120583E4F3F872E878C899D898E1B89
:101660009F0BFC01E058FE4FFD87EC871E821D8218
:101670001C821B8287E0682E712C412C512C212C5E
:10168000312CFF81F7FD1EC0EE85FF85849190E02F
:10169000062C02C0959587950A94E2F780FF08C052
:1016A000088519859701A701B6018D819E8107C024
:1016B0000A851B859701A701B6018B819C818A0D44
:1016C0009B1D20C0FF81F03CF0F0EC85FD858491EE
:1016D00090E0062C02C0959587950A94E2F780FF6A
:1016E00009C0088519859701A701B601C501820DBA
:1016F000931D08C00A851B859701A701B601C50186
:10170000840D951D4ADF280C391C480C591CF1E04A
:101710006F1A71082B813C81280D391D3C832B8366
:101720008D819E81880D991D9E838D839FEF691603
:10173000790609F0A6CFEE89FF893197FF8BEE8BF2
:1017400029813A812E0D3F1D3A832983EF2B09F021
:1017500073CF67960FB6F894DEBF0FBECDBFDF9193
:10176000CF911F910F91FF90EF90DF90CF90BF909E
:10177000AF909F908F907F906F905F904F903F9031
:101780002F9008954F925F926F927F928F929F92C7
:10179000AF92BF92CF92DF92EF92FF920F931F937F
:1017A000CF93DF93EC016B014A013901102F88E0E0
:1017B000089F500111242701F20101912F010023FC
:1017C000B1F020913D0630913E06CE0108962817D3
:1017D000390720F4CA0CDB1CC1E0D0E0E12E9301F4
:1017E000A401B601CE01F0DECA0DDB1DE5CFDF910D
:1017F000CF911F910F91FF90EF90DF90CF90BF900E
:10180000AF909F908F907F906F905F904F900895D2
:101810006F927F928F929F92AF92BF92CF92DF9200
:10182000EF92FF920F93CF93DF9300D000D0CDB70C
:10183000DEB76C015B014A013901C70119821A82C6
:101840001B821C824AE0BE016F5F7F4F0E944A44A8
:10185000CE0101967C019301A401B501C60192DF7E
:101860000F900F900F900F90DF91CF910F91FF90FD
:10187000EF90DF90CF90BF90AF909F908F907F9030
:101880006F9008950F931F9320913B0630913C0673
:1018900060913D0670913E068C0140E050E080E092
:1018A00090E008DE1F910F9108956F927F928F92C2
:1018B0009F92AF92BF92CF92DF92EF92FF920F93DF
:1018C000CF93DF936C01EB017A0159014C01840E37
:1018D000951EB401BBDDBE01CE01C8DD8CE2F0DC9B
:1018E000612C712C6E147F0431F0C5011CDD8FEF6B
:1018F000681A780AF7CF023008F43EC0B401C60176
:10190000A5DDCE010196BC01B1DD8CE2D9DC612CF4
:10191000712C6E147F0431F0C50105DD8FEF681A5C
:10192000780AF7CF023041F1B401C6018FDDCE0154
:101930000296BC019BDD8CE2C3DC612C712C6E1421
:101940007F0431F0C501EFDC8FEF681A780AF7CF1A
:10195000033091F0B401C60179DDCE010396BC01DC
:1019600085DD8CE2ADDCC0E0D0E0CE15DF0521F0F6
:10197000C501D9DC2196F9CFDF91CF910F91FF906E
:10198000EF90DF90CF90BF90AF909F908F907F901F
:101990006F9008956F927F928F929F92AF92BF92B5
:1019A000CF92DF92EF92FF920F93CF93DF93EC01F0
:1019B0006B017A015901BC0149DD46018E0C9F1C67
:1019C000B401C60153DD8CE27BDC612C712C6E14FA
:1019D0007F0431F0C501A7DC8FEF681A780AF7CFD2
:1019E000023008F43EC0CE010196BC012FDDB401E7
:1019F000C6013CDD8CE264DC612C712C6E147F042A
:101A000031F0C50190DC8FEF681A780AF7CF023009
:101A100041F1CE010296BC0119DDB401C60126DDFB
:101A20008CE24EDC612C712C6E147F0431F0C50108
:101A30007ADC8FEF681A780AF7CF033091F0CE0185
:101A40000396BC0103DDB401C60110DD8CE238DC75
:101A5000C0E0D0E0CE15DF0521F0C50164DC2196A1
:101A6000F9CFDF91CF910F91FF90EF90DF90CF9062
:101A7000BF90AF909F908F907F906F9008956F92DE
:101A80007F928F929F92AF92BF92CF92DF92EF920E
:101A90000F931F93CF93DF936C015B01EA01390130
:101AA00048010E2D940101DFB301615071096A0DE7
:101AB0007B1D9401AE01C601F8DE9401A301B501BE
:101AC000C60168DFCE0101979401A301B5018C0D19
:101AD0009D1D60DFDF91CF911F910F91EF90DF90FF
:101AE000CF90BF90AF909F908F907F906F90089510
:101AF000EF92FF920F931F93CF93DF93EB018A0135
:101B00007901BC01640F751FA1DCBE01CE01AEDC02
:101B10008CE2D6DBC0E0D0E0C017D10721F0C701CE
:101B200002DC2196F9CFDF91CF911F910F91FF90A9
:101B3000EF900895EF92FF920F931F93CF93DF934F
:101B4000EB018A017901BC0181DCBE01600F711FCC
:101B5000CE018CDC8CE2B4DBC0E0D0E0C017D10752
:101B600021F0C701E0DB2196F9CFDF91CF911F91E2
:101B70000F91FF90EF9008952F923F924F925F92B6
:101B80006F927F928F929F92AF92BF92CF92DF928D
:101B9000EF92FF920F931F93CF93DF9300D000D06B
:101BA00000D0CDB7DEB76C017B015A0139012801A5
:101BB000261B370B3A8329838A01081B190B17FF51
:101BC00003C0119501951109CA14DB0420F02224E9
:101BD0002A94322C03C022242394312C89819A81A7
:101BE0009E838D8397FF05C09195819591099E8372
:101BF0008D832D813E813195219531093C832B8345
:101C0000E614F70428F08FEF9FEF9A83898304C0CE
:101C100021E030E03A83298348018D819E81881A32
:101C2000990AA201B701C6013DDCC401880F991FC2
:101C30002B813C818217930764F0CA14DB0499F06E
:101C40002D813E81821A930AC20CD31C08171907F2
:101C500044F3E614F70439F0800E911E89819A81CD
:101C6000E80EF91EDECF26960FB6F894DEBF0FBE43
:101C7000CDBFDF91CF911F910F91FF90EF90DF903B
:101C8000CF90BF90AF909F908F907F906F905F901C
:101C90004F903F902F900895AF92BF92CF92DF92D6
:101CA000EF92FF920F931F93CF93DF937C016B0111
:101CB000EA01590198011CDFB501615071096C0DF1
:101CC0007D1D9801AE01C70113DF9801A501B60182
:101CD000C70130DFCE0101979801A501B6018E0D35
:101CE0009F1DDF91CF911F910F91FF90EF90DF909B
:101CF000CF90BF90AF901ECF2F923F924F925F92A6
:101D00006F927F928F929F92AF92BF92CF92DF920B
:101D1000EF92FF920F931F93CF93DF931C012B0140
:101D2000690150E000271127041B150BC1E0D0E02A
:101D3000C41BD50BCC0FDD1FE12CF12CA6015701E4
:101D4000A40CB51CB5013101601A710AC301AADBEC
:101D5000A601B5014801820C931CC401A3DBA601B6
:101D60005201AE18BF08B501C4019CDBA601B50144
:101D7000C30198DBEC16FD06B4F08FEFE81AF80A01
:101D8000C701880F991F01968C0F9D1F22273327AB
:101D9000201B310BE216F30639F40C171D074CF02B
:101DA000C0E0D0E001C0CE010C171D0714F0EC011B
:101DB000C5CF0F5F1F4F9801220F331F2F5F3F4F7B
:101DC000820F931F1016110694F7DF91CF911F9188
:101DD0000F91FF90EF90DF90CF90BF90AF909F90CA
:101DE0008F907F906F905F904F903F902F900895CD
:101DF0004F925F926F927F928F929F92AF92BF921B
:101E0000CF92DF92EF92FF920F931F93CF93DF93C6
:101E1000EC015B014A01390128018601ADDE970121
:101E2000A201B301C401A8DE9501AE01B701C20150
:101E3000A3DEDF91CF911F910F91FF90EF90DF9084
:101E4000CF90BF90AF909F908F907F906F905F905A
:101E50004F900895CF93C82F8A3011F48DE0FADFA8
:101E60005D9BFECFCCB980E090E0CF910895CF92FA
:101E7000DF92EF92FF920F931F93CF93DF93CDB733
:101E8000DEB761970FB6F894DEBF0FBECDBF90E00E
:101E90008A30910508F0EFC1FC01EA5BFF4F0C941A
:101EA0003244A8958AE0EFE3F1E0DE01119601905B
:101EB0000D928A95E1F7CE0101967C0101E02FE1B8
:101EC00030E04FEF5FEF63E270E08AE090E05ADCD1
:101ED000A895E091DD068E2F90E08830910508F0FE
:101EE000CAC1FC01E05BFF4F0C943244B9EAEB2E0F
:101EF000B5E0FB2E04C0A4EAEA2EA5E0FA2E02E02B
:101F00002FE130E04FEF5FEF6EE170E08BEE90E09D
:101F1000B1C1FCE7EF2EF5E0FF2E72C1E2E7EE2E35
:101F2000E5E0FE2E6DC178E6E72E75E0F72E68C17C
:101F3000A89588E0E9E4F1E0DE01119601900D92A8
:101F40008A95E1F786E0E6EAF1E0DE011C96019071
:101F50000D928A95E1F7CE0101967C0101E02FE117
:101F600030E04FEF5FEF64E170E084E190E00ADC85
:101F7000CE010C967C012FE130E04FEF5FEF68E27D
:101F800070E08EE190E0FEDBA89580918B0602C1A7
:101F9000A89587E0E1E5F1E0DE01119601900D9250
:101FA0008A95E1F786E0E6EAF1E0DE011C96019011
:101FB0000D928A95E1F7CE0101967C0101E02FE1B7
:101FC00030E04FEF5FEF64E170E084E190E0DADB56
:101FD000CE010C967C012FE130E04FEF5FEF68E21D
:101FE00070E08EE190E0CEDBA89580919206D2C0A1
:101FF000A89587E0E8E5F1E0DE01119601900D92E9
:102000008A95E1F7CE0101967C0101E02FE130E0F5
:102010004FEF5FEF63E270E089E190E0B3DBA895FA
:102020002FE130E04FEF5FEF6EE170E08EEE90E079
:10203000A9DB40EEC42E47E0D42E51E6E52EF12C6C
:102040000EE110E021E630E04AE050E067E570E0A4
:1020500084E190E0CDDE06E311E021E630E042E2EB
:1020600051E067E570E08CE291E0C2DE60EAE62EC6
:10207000F12C0EE110E020EA30E04AE050E06AEA9C
:1020800070E084E190E0B4DE06E311E020EA30E0A5
:1020900042E251E06AEA70E08CE291E0A9DEEBC036
:1020A000A8958BE0EFE5F1E0DE01119601900D922D
:1020B0008A95E1F7CE0101967C0101E02FE130E045
:1020C0004FEF5FEF63E270E08FE090E05BDBA8959D
:1020D0008091E7065FC0A89586E0EAE6F1E0DE01C0
:1020E0001C9601900D928A95E1F78AE0E0E7F1E015
:1020F000DE01119601900D928A95E1F7CE010C96C2
:102100007C0101E02FE130E04FEF5FEF64E170E030
:1021100089E190E037DBCE0101967C012FE130E0D0
:102120004FEF5FEF63E270E08FE090E02BDBA8956C
:102130008091DC062FC0A89586E0EAE6F1E0DE019A
:10214000119601900D928A95E1F785E0EAE7F1E0BA
:10215000DE011C9601900D928A95E1F7CE01019661
:102160007C0101E02FE130E04FEF5FEF64E170E0D0
:1021700089E190E007DBCE010C967C012FE130E095
:102180004FEF5FEF63E270E08FE190E0FBDAA8953C
:102190008091D906813059F110F53AE9E32E35E006
:1021A000F32E2EC0A89588E0E3EEF1E0DE01119653
:1021B00001900D928A95E1F7CE0101967C0101E034
:1021C0002FE130E04FEF5FEF63E270E08FE090E0EF
:1021D000D9DAA89580919906813049F018F08230BB
:1021E00059F049C020E6E22E25E0F22E09C090E920
:1021F000E92E95E0F92E04C086E8E82E85E0F82E59
:1022000001E030C0A8958BE0EFE7F1E0DE01119628
:1022100001900D928A95E1F785E0EAE8F1E0DE01B0
:102220001C9601900D928A95E1F7CE0101967C01F2
:1022300001E02FE130E04FEF5FEF64E170E08AE012
:1022400090E0A0DACE010C967C012FE130E04FEF58
:102250005FEF68E270E08EE190E094DAA895CE013D
:1022600001967C012FE130E04FEF5FEF6EE170E00F
:1022700086EE90E087DA61960FB6F894DEBF0FBE67
:10228000CDBFDF91CF911F910F91FF90EF90DF9025
:10229000CF900895CF93DF9300D000D0CDB7DEB7B5
:1022A0008091630080FD21C01C821B821A821982EA
:1022B000BE016F5F7F4FCE0103960E9495428B81D6
:1022C0009C81853C994088F0A89589819A81843CBD
:1022D000994058F4A89589819A818D3D954028F0C0
:1022E000A89581E080938406A8950F900F900F9099
:1022F0000F90DF91CF910895CF93DF9300D000D05E
:10230000CDB7DEB7A8958091630080FD23C01C8205
:102310001B821A821982BE016F5F7F4FCE01039626
:102320000E9495428B819C81853C994098F08981DF
:102330009A81843C994070F489819A818D3D9540C1
:1023400048F0109284068FE19EE40197F1F700C0F7
:102350000000A8950F900F900F900F90DF91CF91F4
:102360000895CF92DF92EF92FF920F931F93A8955B
:1023700080918406811140C0A8950FE110E02CE403
:1023800030E04EE650E06CE870E089E690E005D978
:1023900020E038EF48E264EB70E080EA90E0ACDCEB
:1023A00020E038EF47E264EB70E080EA90E0A4DCE4
:1023B00020E038EF4BE264EB70E080EA90E09CDCD8
:1023C00020E038EF45E264EB70E080EA90E094DCD6
:1023D00000E018EF23E230E045E050E065EA70E00D
:1023E00086E990E0DAD823E230E045E050E065EAA3
:1023F00070E085EA90E0D1D880918406813009F0C0
:102400003EC0A8950FE110E02CE430E04EE650E02D
:102410006CE870E089E690E0C0D820EE37E048E252
:1024200064EB70E080EA90E067DC20EE37E047E2A2
:1024300064EB70E080EA90E05FDC20EE37E04BE296
:1024400064EB70E080EA90E057DC20EE37E045E294
:1024500064EB70E080EA90E04FDC80EEC82E87E00D
:10246000D82E94EBE92EF12C07EB10E028EC30E0AD
:1024700044E950E060EA70E084E990E0B9DC1F9143
:102480000F91FF90EF90DF90CF900895EF92FF9221
:102490000F931F93CF93DF93CDB7DEB764970FB63B
:1024A000F894DEBF0FBECDBFA8950FEF1FEF21E45C
:1024B00030E04FE550E065E070E085E090E0ECDB77
:1024C000A89521E430E04FE550E06BE470E085E052
:1024D00090E0E2DB2BE430E04FE550E061E970E0B2
:1024E00085E090E0D9DB89E0EFE8F1E0DE011196CC
:1024F00001900D928A95E1F785E0EAE8F1E0DE01CE
:10250000509601900D928A95E1F7CE0101967C01DB
:1025100001E02FE130E04FEF5FEF60E570E082E136
:1025200090E030D9CE0140967C012FE130E04FEFB2
:102530005FEF6AE570E083E290E024D90FEF1FEFD0
:1025400021E430E04FE550E065E070E08CED90E094
:10255000A3DB21E430E04FE550E06BE470E08CED6C
:1025600090E09ADB2BE430E04FE550E061E970E069
:102570008CED90E091DB86E0E8E9F1E0DE011A966F
:1025800001900D928A95E1F7CE0101967C0101E060
:102590002FE130E04FEF5FEF60E570E08BEE90E011
:1025A000F1D8CE010A967C012FE130E04FEF5FEFCA
:1025B0006AE570E08CEF90E0E5D88EE4E82E83E0E9
:1025C000F82E2FE130E04FEF5FEF66EE70E08AE02B
:1025D00090E0D8D8C6DE8091850649DC64960FB6B7
:1025E000F894DEBF0FBECDBFDF91CF911F910F9149
:1025F000FF90EF900895EF92FF920F93CF93DF93A8
:10260000CDB7DEB7C458D1090FB6F894DEBF0FBE00
:10261000CDBF9AE0EFE3F1E0DE01AA59BF4F019090
:102620000D929A95E1F79EE0EEE9F1E0DE015E960B
:1026300001900D929A95E1F79EE0ECEAF1E0DE015F
:10264000509601900D929A95E1F79CE0EAEBF1E04B
:10265000DE01AB5BBF4F01900D929A95E1F79BE0D5
:10266000EFE5F1E0DE01AF5ABF4F01900D929A9570
:10267000E1F796E0EAE6F1E0DE01A158BF4F0190F4
:102680000D929A95E1F79AE0E0E7F1E0DE01A45AB5
:10269000BF4F01900D929A95E1F79DE0E6ECF1E0D5
:1026A000DE019C9601900D929A95E1F79FE0E3ED93
:1026B000F1E0DE01119601900D929A95E1F799E013
:1026C000E2EEF1E0DE01A059BF4F01900D929A9524
:1026D000E1F79CE0EBEEF1E0DE01D99601900D927E
:1026E0009A95E1F796E0E7EFF1E0DE01A758BF4FDA
:1026F00001900D929A95E1F7A89590E08A309105A6
:1027000008F06BC0FC01E85AFF4FCE010C94324434
:102710008A599F4F7C0102E02FE130E04FEF5FEFDD
:1027200062E870E030C04E9626C0409624C08B5BB5
:102730009F4F21C08F5A9F4F1EC081589F4F7C01D1
:1027400002E02FE130E04FEF5FEF6EE670E088E2ED
:1027500090E018D8CE01845A9F4F7C012FE130E0E1
:102760004FEF5FEF67E870E08FE090E034C08C9649
:1027700002C080599F4F7C0102E02FE130E04FEF13
:102780005FEF68E770E088E090E025C001967C018B
:1027900002E02FE130E04FEF5FEF68E770E082E0AA
:1027A00090E019C0C9967C0102E02FE130E04FEFC4
:1027B0005FEF6EE670E084E190E00E94C20BCE0114
:1027C00087589F4F7C012FE130E04FEF5FEF67E8C4
:1027D00070E08CE390E00E94C20BCC57DF4F0FB645
:1027E000F894DEBF0FBECDBFDF91CF910F91FF9068
:1027F000EF900895CF92DF92EF92FF920F931F9385
:10280000A89500EE17E021E430E048EC50E06AEAD9
:1028100070E085E090E00E94CD0A0FEF1FEF21E409
:1028200030E048EC50E063E270E085E090E034DABC
:1028300084E7E82E83E0F82E01E02FE130E040EE5F
:1028400057E06CE370E088E290E00E94C20B0FEF6B
:102850001FEF20E530E040E550E065E070E08BEEF2
:1028600090E01ADA90EEC92E97E0D92E24E1E22EFC
:10287000F12C03E111E026E430E041E351E066E4AD
:1028800070E085EF90E0B4DA37E1E32EF12C24E438
:1028900030E04FE251E064E470E087EF90E0A8DAC6
:1028A0000FEF1FEF20E530E040E550E064E670E018
:1028B0008BEE90E0F1D945EAE42EF12C03E111E032
:1028C00023E730E041E351E063E770E085EF90E01B
:1028D0008FDA53EAE52EF12C25E730E04FE251E0A4
:1028E00065E770E087EF90E083DA68EBE62E65E05D
:1028F000F62E02E020EE37E040E050E068EC70E0B9
:102900008DE290E00E94C20B1F910F91FF90EF901B
:10291000DF90CF900895CF92DF92EF92FF920F93C6
:102920001F93CF93DF93CDB7DEB765970FB6F894BB
:10293000DEBF0FBECDBFA8958FE0E3EDF1E0DE0175
:10294000119601900D928A95E1F786E0EDEFF1E0A6
:10295000DE01509601900D928A95E1F700EE17E0A6
:1029600021E430E048EC50E06AEA70E085E090E075
:102970000E94CD0A0FEF1FEF21E430E048EC50E059
:1029800063E270E085E090E087D9CE0101967C019A
:1029900001E02FE130E040EE57E06CE370E088E2C8
:1029A00090E00E94C20B0FEF1FEF20E530E040E502
:1029B00050E065E070E08BEE90E06ED980EEC82EBE
:1029C00087E0D82E94E1E92EF12C03E111E026E412
:1029D00030E041E351E066E470E085EF90E008DA32
:1029E00027E1E22EF12C24E430E04FE251E064E4F0
:1029F00070E087EF90E0FCD90FEF1FEF20E530E0AB
:102A000040E550E064E670E08BEE90E045D935EAB1
:102A1000E32EF12C03E111E023E730E041E351E044
:102A200063E770E085EF90E0E3D943EAE42EF12C10
:102A300025E730E04FE251E065E770E087EF90E096
:102A4000D7D9CE0140967C0102E020EE37E040E08D
:102A500050E068EC70E08DE290E00E94C20B659659
:102A60000FB6F894DEBF0FBECDBFDF91CF911F919F
:102A70000F91FF90EF90DF90CF900895CF92DF926B
:102A8000EF92FF920F931F93A89500EE17E021E4B9
:102A900030E048EC50E06AEA70E085E090E00E94A7
:102AA000CD0A0FEF1FEF21E430E048EC50E063E285
:102AB00070E085E090E0F0D88FE4E82E85E0F82E15
:102AC00001E02FE130E040EE57E06CE370E088E297
:102AD00090E00E94C20B0FEF1FEF20E530E040E5D1
:102AE00050E065E070E08BEE90E0D6D890EEC92E15
:102AF00097E0D92E24E1E22EF12C03E111E026E447
:102B000030E041E351E066E470E085EF90E070D999
:102B100037E1E32EF12C24E430E04FE251E064E4AD
:102B200070E087EF90E064D90FEF1FEF20E530E011
:102B300040E550E064E670E08BEE90E0ADD845EA09
:102B4000E42EF12C03E111E023E730E041E351E012
:102B500063E770E085EF90E04BD953EAE52EF12C66
:102B600025E730E04FE251E065E770E087EF90E065
:102B70003FD969ECE62E65E0F62E02E020EE37E064
:102B800040E050E068EC70E08DE290E00E94C20B03
:102B90001F910F91FF90EF90DF90CF900895CF930A
:102BA000DF9300D000D0CDB7DEB78091630080FD09
:102BB00057C01C821B821A821982BE016F5F7F4F31
:102BC000CE0103960E9495428B819C818431954071
:102BD00068F489819A81843A964040F489819A8187
:102BE0008D32914018F082E08093A7068B819C8102
:102BF0008937954090F08B819C81843C994068F4A2
:102C000089819A81843A964040F489819A818D32F3
:102C1000914018F083E08093A7068B819C818932D4
:102C20009A4068F089819A8184379E4040F4898176
:102C30009A81813D974018F081E08093A7068B81AF
:102C40009C81863F994060F48B819C8181349640C1
:102C500038F089819A81813D974010F01092A70643
:102C60008091A7060F900F900F900F90DF91CF915A
:102C70000895CF92DF92EF92FF920F931F93CF931D
:102C8000DF9300D000D000D0CDB7DEB7A89586E0A6
:102C9000EDEFF1E0DE01119601900D928A95E1F7DA
:102CA00000EE17E021E430E048EC50E06AEA70E022
:102CB00085E090E00E94CD0A0FEF1FEF21E430E0A5
:102CC00048EC50E063E270E085E090E00E944C0E3A
:102CD00020E530E040E550E065E070E08BEE90E00C
:102CE0000E944C0EF0EECF2EF7E0DF2EA4E1EA2E8C
:102CF000F12C03E111E026E430E041E351E066E429
:102D000070E085EF90E074D8B7E1EB2EF12C24E46D
:102D100030E04FE251E064E470E087EF90E068D883
:102D20000FEF1FEF20E530E040E550E064E670E093
:102D30008BEE90E00E944C0E15EAE12EF12C03E19F
:102D400011E023E730E041E351E063E770E085EF15
:102D500090E04ED883EAE82EF12C25E730E04FE2F0
:102D600051E065E770E087EF90E042D8CE01019630
:102D70007C0102E020EE37E040E050E068EC70E0DB
:102D80008CE390E00E94C20B80918506811148C0BF
:102D9000E091DD068E2F90E08830910508F040C06C
:102DA000FC01EE59FF4F0C943244E9EAEE2EE5E0C7
:102DB000FE2E04C074EAE72E75E0F72E02E02FE144
:102DC00030E04FEF5FEF65E070E086E490E026C012
:102DD0006AE9E62E65E0F62E18C050E9E52E55E0CA
:102DE000F52E13C046E8E42E45E0F42E0EC03CE775
:102DF000E32E35E0F32E09C022E7E22E25E0F22E85
:102E000004C098E6E92E95E0F92E02E02FE130E0CB
:102E10004FEF5FEF65E070E08EE190E00E94C20B43
:102E200080918506813001F580918B06813069F0B3
:102E300038F08230C9F416E8E12E15E0F12E09C011
:102E40008AE9E82E85E0F82E04C000E9E02E05E0CE
:102E5000F02E02E02FE130E04FEF5FEF65E070E031
:102E60008EE190E00E94C20B80918506823001F5D0
:102E700080919206813069F038F08230C9F4F6E82A
:102E8000EF2EF5E0FF2E09C0BAE9EB2EB5E0FB2EE0
:102E900004C0A0E9EA2EA5E0FA2E02E02FE130E01E
:102EA0004FEF5FEF65E070E08EE190E00E94C20BB3
:102EB00080918506843001F58091E706813069F0C4
:102EC00038F08230C9F466E8E62E65E0F62E09C0D7
:102ED000EAE9EE2EE5E0FE2E04C070E9E72E75E08B
:102EE000F72E02E02FE130E04FEF5FEF65E070E09A
:102EF0008EE190E00E94C20B80918506853001F53D
:102F00008091DC06813069F038F08230C9F436E80F
:102F1000E32E35E0F32E09C05AE9E52E55E0F52EF3
:102F200004C040E9E42E45E0F42E02E02FE130E059
:102F30004FEF5FEF65E070E08EE190E00E94C20B22
:102F400080918506863001F58091D906813069F03F
:102F500038F08230C9F486E8E82E85E0F82E09C002
:102F60002AE9E22E25E0F22E04C090E9E92E95E050
:102F7000F92E02E02FE130E04FEF5FEF65E070E007
:102F80008EE190E00E94C20B26960FB6F894DEBF49
:102F90000FBECDBFDF91CF911F910F91FF90EF90AA
:102FA000DF90CF900895EF92FF920F931F9380913F
:102FB0007D0690917E060A97A8F4809154068111AF
:102FC0000CC00FE110E02CE330E044E650E06BE48D
:102FD00070E08EE690E00E94CD0A81E08093540676
:102FE0001092860680917D0690917E060A978A351A
:102FF0009105A8F48091860681110CC00FE110E0C4
:103000002CE330E044E650E06BE470E08EE690E0C4
:103010000E94CD0A81E0809386061092540680912A
:103020007D0690917E0684369105E8F081329340CA
:1030300030F087EE93E090937E0680937D0680913A
:103040008606813061F40FE110E02CE330E044E6C5
:1030500050E06BE470E08EE690E00E94CD0A1092A2
:1030600086061092540680918406813079F4E090AF
:103070007D06F0907E0603E02FE130E04FEF5FEF3A
:1030800064E670E082E890E00E94080C809184067B
:1030900081110FC0E0907D06F0907E0603E02FE1E5
:1030A00030E040E058EF64E670E082E890E00E9493
:1030B000080C1F910F91FF90EF900895EF92FF92EF
:1030C0000F931F938091AB069091AC060A97A8F4DA
:1030D00080917C06811111C00FE110E028E230E000
:1030E00048E550E06FEA70E088E090E00E94CD0A89
:1030F00081E080937C061092DA068091AB06909175
:10310000AC0684369105D8F480917D0690917E06B8
:103110000A97A8F08091DA06811111C00FE110E042
:1031200028E230E048E550E06FEA70E088E090E0A7
:103130000E94CD0A81E08093DA0610927C0680918D
:10314000AB069091AC0684369105E8F0813293404D
:1031500030F087EE93E09093AC068093AB068091BD
:10316000DA06813061F40FE110E028E230E048E552
:1031700050E06FEA70E088E090E00E94CD0A109283
:10318000DA0610927C06E090AB06F090AC0602E006
:103190002FE130E04FEF5FEF6EEB70E08EE190E0FB
:1031A0000E94080C1F910F91FF90EF900895EF92ED
:1031B000FF920F931F9380919A068A30A8F4809112
:1031C000830681110CC00FE110E024E230E04AE5F3
:1031D00050E064E670E088E090E00E94CD0A81E073
:1031E000809383061092960680919A068A508A35BB
:1031F000A8F48091960681110CC00FE110E024E242
:1032000030E04AE550E064E670E088E090E00E943B
:10321000CD0A81E0809396061092830680919A06EB
:103220008436A1F480919606813061F40FE110E0BC
:1032300024E230E04AE550E064E670E088E090E0A7
:103240000E94CD0A109283061092960680919A06EB
:10325000843618F084E680939A06E0909A06F12C62
:1032600002E02FE130E04FEF5FEF6EE670E084E1C7
:1032700090E00E94080C8091E8068A30A8F48091C2
:10328000E306811111C00FE110E024E230E04AE5CD
:1032900050E064E670E08FED90E00E94CD0A81E09E
:1032A0008093E3061092AD068091E8068A508A3535
:1032B000A8F48091AD06811111C00FE110E024E265
:1032C00030E04AE550E064E670E08FED90E00E9467
:1032D000CD0A81E08093AD061092E3068091E80666
:1032E000843629F41092E3061092AD0602C08436AB
:1032F00018F084E68093E806E090E806F12C02E0FE
:103300002FE130E04FEF5FEF6EE670E089EE90E086
:103310000E94080C1F910F91FF90EF9008957F92EB
:103320008F929F92AF92BF92CF92DF92EF92FF92D5
:103330000F931F93CF93DF93EC016B015A01490167
:10334000702EA89580915706909158060A97A8F478
:103350008091DE06811111C00FE110E02EE130E016
:1033600044E650E065507109CE0144970E94CD0AB1
:1033700081E08093DE061092A0068091570690911E
:1033800058060A978A359105C0F48091A0068111EC
:1033900014C00FE110E02EE130E044E650E0B60149
:1033A00065507109CE0144970E94CD0A81E0809357
:1033B000A0061092DE0610927F068091570690912B
:1033C000580684369105C0F080917F06811114C0A3
:1033D0000FE110E02EE130E044E650E0B601655028
:1033E0007109CE0144970E94CD0A81E080937F0647
:1033F0001092A0061092DE06E0905706F090580654
:10340000072D9401A501B601CE010E94080CA895D4
:10341000DF91CF911F910F91FF90EF90DF90CF90B0
:10342000BF90AF909F908F907F900895CF92DF9242
:10343000EF92FF920F931F938FE190E00E94420C56
:10344000A89500EE17E021E430E048EC50E06AEA8D
:1034500070E085E090E00E94CD0A0FEF1FEF21E4BD
:1034600030E048EC50E063E270E085E090E00E94DC
:103470004C0E8EE3E82E83E0F82E01E02FE130E0E1
:1034800040EE57E06CE370E088E290E00E94C20BEF
:103490000FEF1FEF20E530E040E550E065E070E021
:1034A0008BEE90E00E944C0E90EEC92E97E0D92E44
:1034B00024E1E22EF12C03E111E026E430E041E3C7
:1034C00051E066E470E085EF90E00E94F80E37E18D
:1034D000E32EF12C24E430E04FE251E064E470E0AC
:1034E00087EF90E00E94F80E0FEF1FEF20E530E02D
:1034F00040E550E064E670E08BEE90E00E944C0EF8
:1035000045EAE42EF12C03E111E023E730E041E34A
:1035100051E063E770E085EF90E00E94F80E53EA17
:10352000E52EF12C25E730E04FE251E065E770E051
:1035300087EF90E00E94F80E68EBE62E65E0F62E2D
:1035400002E020EE37E040E050E068EC70E08DE211
:1035500090E00E94C20B8FE19EE40197F1F700C05A
:1035600000001F910F91FF90EF90DF90CF90089592
:10357000A8958BED92E00E944D47813071F4A49A9A
:1035800080E185BBA8952FEF82E597E02150804030
:103590009040E1F700C0000015BAA8950895A895DD
:1035A0008BED92E00E944D47813021F5A49A80E195
:1035B00085BB2FEF32E597E0215030409040E1F796
:1035C00000C00000A89515BA2FEF32E597E0215012
:1035D00030409040E1F700C00000A89585BB2FEF78
:1035E00032E587E0215030408040E1F700C0000024
:1035F000A89515BA0895A8958BED92E00E944D47C5
:10360000813009F048C0A49A80E185BBA8952FEFCE
:1036100032E597E0215030409040E1F700C00000D3
:10362000A89515BAA8952FEF32E597E021503040C4
:103630009040E1F700C00000A89585BBA8952FEF4A
:1036400032E597E0215030409040E1F700C00000A3
:10365000A89515BAA8952FEF32E597E02150304094
:103660009040E1F700C00000A89585BB2FEF32E540
:1036700087E0215030408040E1F700C00000A8956D
:1036800015BA9FEF22E537E0915020403040E1F736
:1036900000C00000A89508951092E806BC9A809199
:1036A000E806880F81BF10929A06139A80919A06B5
:1036B000880F809386009FDF8DE490E09093E00672
:1036C0008093DF060895A89510929B0610928F06AE
:1036D000109252061092B00610928C06109282063A
:1036E00010929C06109295061092AA06109253060C
:1036F000A8958CED92E00E94554790939106809397
:103700009006A8958091850681112AC0A895E09120
:10371000DD068E2F90E08830910510F5FC01E6590A
:10372000FF4F4EE150E00C9432446CEB72E014C059
:103730006EE972E011C060E872E00EC062E672E00D
:103740000BC064E472E008C066E272E005C068E0A5
:1037500072E002C06AEE71E08DE596E00E943D479E
:10376000A895809185068130D1F4A89580918B062B
:10377000813069F038F0823091F44EE150E060E938
:1037800071E009C04EE150E06CEC71E004C04EE124
:1037900050E06EEA71E08DE596E00E943D47A89505
:1037A000809185068230D1F4A8958091920681306F
:1037B00069F038F0823091F44EE150E066E371E058
:1037C00009C04EE150E062E771E004C04EE150E014
:1037D00064E571E08DE596E00E943D47A8958091F3
:1037E00085068430C9F48091E706813069F038F0AD
:1037F000823091F44EE150E06CED70E009C04EE192
:1038000050E068E171E004C04EE150E06AEF70E022
:103810008DE596E00E943D47A8958091850685300C
:10382000C9F48091DC06813069F038F0823091F47F
:103830004EE150E062E870E009C04EE150E06EEB0E
:1038400070E004C04EE150E060EA70E08DE596E083
:103850000E943D47A895809185068630C9F48091E5
:10386000D906813069F038F0823091F44EE150E0B1
:1038700068E270E009C04EE150E064E670E004C028
:103880004EE150E066E470E08DE596E00E943D4731
:10389000A89587EC90E00197F1F700C000008091B7
:1038A0005D0690915E0690934F0680934E06809140
:1038B0005F069091600690939F0680939E0680918C
:1038C00061068093E5068091630680938A06809165
:1038D00065068093B2068091670680938906809181
:1038E00069068093980680916B0680939706809175
:1038F0006D0680934A0680916F06909170069093B2
:10390000D6068093D506809171068093B10680918A
:103910008506873021F48091730680938506809117
:103920007506909176069093D4068093D306809185
:1039300077069091780690935C0680935B06809161
:10394000790690917A069093810680938006A895D7
:1039500008958091B006811117C020918906809149
:103960007D0690917E06821B9109029768F482E39E
:103970008093E80681E08093B00680938206809170
:10398000B206811101C0F4DD2091890630E060911A
:10399000E5064091E1065091E206649FC001659FF3
:1039A000900D11246AE070E00E941E44620F731FA4
:1039B00070934D0660934C069091E80640914E0638
:1039C00050914F064617570720F450934D064093E9
:1039D0004C0680919806891710F48093E806809130
:1039E0007D0690917E062817390720F04817590761
:1039F00028F155C02091AA062111F8CF8417950708
:103A0000A8F760914C0670914D062091E806861744
:103A1000970750F42F5F253618F42093E806E6CF79
:103A200024E62093E80687C0222319F02150209332
:103A3000E8062091E8062223C9F27DC02091E8061D
:103A4000222319F021502093E806841B950B06973A
:103A500068F08091E8068A3010F41092E8068091B0
:103A6000E8068A3018F08A508093E8068091530661
:103A7000811106C094DD81E0809395068093530602
:103A80002091590630915A068091900690919106A6
:103A90008217930720F400DE81E0809384068091F2
:103AA0008C0681114FC04091D3065091D40680916D
:103AB000890690E08417950708F044C0E0917D06E0
:103AC000F0917E064E175F0729F481E08093AA06E5
:103AD00080939C068091AA068130A1F560915506DD
:103AE0007091560620915B0630915C066217730751
:103AF00078F48091E806E417F50728F48F5F85369F
:103B000028F084E603C0882319F081508093E806EA
:103B100026173707B8F41092AA068091E106909113
:103B2000E206821B930B9093E2068093E10681E00C
:103B300080938C0608954817590708F0B0CF20915C
:103B4000E80680CF08958091B006811117C080915A
:103B5000890690E020917D0630917E0682179307BA
:103B600068F482E38093E80681E08093B006809356
:103B700082068091B206811101C0FADCE0918906CB
:103B8000F0E04091E5062091E1063091E206429F87
:103B9000C001439F900D11246AE070E00E941E4412
:103BA0006E0F7F1F70934D0660934C069091E80650
:103BB00040914E0650914F064617570720F45093F8
:103BC0004D0640934C0680919806891710F4809317
:103BD000E80620917D0630917E06E217F307D0F4C7
:103BE0008091AA06811116C02417350798F46091B8
:103BF0004C0670914D068091E8062617370728F489
:103C00008F5F853628F084E603C0882319F0815041
:103C10008093E8064217530770F58091E8068150BB
:103C20008093E806241B350B2630310558F08A3086
:103C300010F41092E8068091E8068A3018F08A5055
:103C40008093E80680915306811106C0A8DC81E0CC
:103C500080939506809353062091590630915A0619
:103C600080919006909191068217930720F414DDBD
:103C700081E08093840680918C06811146C040913A
:103C8000D3065091D4068091890690E08417950759
:103C9000E0F5E0917D06F0917E064E175F0729F46E
:103CA00081E08093AA0680939C068091AA068130C9
:103CB00061F5609155067091560620915B06309132
:103CC0005C066217730778F48091E806E417F5073D
:103CD00028F48F5F853628F084E603C0882319F026
:103CE00081508093E8062617370778F41092AA06C9
:103CF0008091E1069091E206821B930B9093E2067D
:103D00008093E10681E080938C06089540918A06B5
:103D10002091570630915806429FC001439F900D55
:103D200011246AE070E00E941E447093AF06609315
:103D3000AE0680919A06853618F084E680939A063E
:103D40009091970680919A06981710F490939A068E
:103D500080919B062091AB063091AC0681110DC07D
:103D60002639310520F484E680939A0606C0263968
:103D7000310519F081E080939B0680919B0640916C
:103D80009E0650919F068130D9F464177507C0F4E0
:103D900080919A062617370770F48F5F981718F0EE
:103DA00080939A0602C090939A0680919A0685366F
:103DB00038F084E603C0882319F0815080939A0676
:103DC0004617570768F52417350770F480919A064F
:103DD0008F5F853608F084E680939A0680919A0674
:103DE000981710F490939A0642175307C8F48091DD
:103DF0009A06882319F0815080939A06C901841B82
:103E0000950B0B9768F080919A068A3010F4109207
:103E10009A0680919A068A3018F08A5080939A0602
:103E2000809198069091E806891710F48093E8062F
:103E30004217530740F48091E8068F5F853608F0FB
:103E400084E68093E806089540918A0620915706FB
:103E500030915806429FC001439F900D11246AE0A3
:103E600070E00E941E447093AF066093AE0680918E
:103E70009A06853618F084E680939A069091970604
:103E800080919A06981710F490939A0680919B0659
:103E9000811111C02091AB063091AC062639310555
:103EA00020F484E680939A0606C02639310519F07D
:103EB00081E080939B0680919B0640919E065091E5
:103EC0009F068130F9F464177507E0F42091AB0682
:103ED0003091AC0680919A062617370770F48F5FF1
:103EE000981718F080939A0602C090939A068091D2
:103EF0009A06853638F084E603C0882319F081508D
:103F000080939A064617570788F52091AB063091A3
:103F1000AC062417350770F480919A068F5F8536BA
:103F200008F084E680939A0680919A06981710F418
:103F300090939A0642175307C8F480919A068823F3
:103F400019F0815080939A06241B350B2B303105D4
:103F500068F080919A068A3010F410929A06809147
:103F60009A068A3018F08A5080939A0608958091B4
:103F70007D0690917E068B35910510F010929A0681
:103F800080919B06811113C08091AB069091AC0685
:103F9000883121E0920720F484E680939A0607C0D6
:103FA0008831914021F0E4DA81E080939B06809192
:103FB0009B06813081F48091AB069091AC06813AEA
:103FC000910518F010929A0608958837910518F413
:103FD0008AE080939A060895CF93C091B206C130CB
:103FE000D9F480918F06811117C08091890690E0E5
:103FF00020917D0630917E062817390768F0809160
:10400000AB069091AC068A55910990935106809326
:104010005006AEDAC0938F0640918A06209157066B
:1040200030915806429FC001439F900D11246AE0D1
:1040300070E00E941E447093AF066093AE068091BC
:104040009A06853618F084E680939A0680919B063E
:10405000811112C08091AB069091AC068C3221E0A8
:10406000920720F484E680939A0606C08C32914031
:1040700019F081E080939B0680919B06C0918F068A
:104080008130A1F5C11124C080919E0690919F06B8
:1040900068177907E8F42091AB063091AC0680915F
:1040A0009A062617370778F48F5F80939A069091C7
:1040B0009706981710F490939A0680919A06853681
:1040C00038F084E603C0882319F0815080939A0663
:1040D0008091890690E00A9720917D0630917E06B6
:1040E0008217930718F486E480939A06C13091F4FE
:1040F00080915006909151060E948703C0939506C7
:104100008091590690915A06CD9720F010925A0648
:104110001092590680919E0690919F062091AE06BE
:104120003091AF068217930740F42091B206211117
:1041300004C08A5591090E948703C0914A06C13084
:10414000F9F48091520681111BC080917D069091F7
:104150007E062091D5063091D606821B930B0597DB
:1041600078F42091B1068091500690915106820F0B
:10417000911D9093510680935006FAD9C093520630
:10418000CF910895BC9A8091E806880F81BF139A59
:1041900080919A06880F8093860080918506811110
:1041A00002C01ADFD6DB80918506813019F41092A7
:1041B0009A06C9DC80918506823019F41092E806CF
:1041C0000BDF80918506833011F40E94CB03809130
:1041D0008506843009F49ADD80918506853009F4DE
:1041E00095DD80918506863009F42EDE8091850666
:1041F000873009F4BCDE80918506893069F48091AE
:10420000AB069091AC060E944C0380919A068635CD
:1042100018F081E080938406089563EC70E08CEBE5
:1042200092E00E94704762EC71E08EEB92E00E9497
:10423000704766E170E080EC92E00E94704766E1B2
:1042400070E082EC92E00E94704761E070E084ECE4
:1042500092E00E947047A8956EE670E086EC92E0CE
:104260000E94704764E670E088EC92E00E9470471C
:1042700064E670E08AEC92E00E94704760E070E0D3
:104280008CEC92E00E947047A89560E070E08EECA4
:1042900092E00E94704760E070E080ED92E00E9442
:1042A000704760E070E082ED92E00E94704760E04D
:1042B00070E084ED92E00E94704760E070E086ED6F
:1042C00092E00E94704760E070E088ED92E00E940A
:1042D0007047A89566EE70E08EE992E00E94704704
:1042E00062EC71E080EA92E00E94704766E170E063
:1042F00082EA92E00E94704766E170E084EA92E010
:104300000E94704761E070E086EA92E00E94704788
:10431000A89563E770E088EA92E00E94704764E63F
:1043200070E08AEA92E00E94704764E670E08CEAEE
:1043300092E00E94704760E070E08EEA92E00E9496
:10434000704760E070E080EB92E00E94704760E0B0
:1043500070E082EB92E00E947047A89560E070E008
:1043600084EB92E00E94704760E070E086EB92E0A0
:104370000E94704760E070E088EB92E00E94704716
:1043800060E070E08AEB92E00E947047A89566EECC
:1043900070E080E892E00E94704762EC71E082E891
:1043A00092E00E94704766E170E084E892E00E942B
:1043B000704766E170E086E892E00E94704761E035
:1043C00070E088E892E00E947047A89563E770E08B
:1043D0008AE892E00E94704764E670E08CE892E020
:1043E0000E94704764E670E08EE892E00E94704799
:1043F00060E070E080E992E00E94704760E070E069
:1044000082E992E00E94704760E070E084E992E007
:104410000E947047A89560E070E086E992E00E94F3
:10442000704760E070E088E992E00E94704760E0C9
:1044300070E08AE992E00E94704760E070E08CE9E9
:1044400092E00E947047A89566E970E082E692E0EB
:104450000E94704768EC70E084E692E00E9470472A
:1044600066E170E086E692E00E94704766E170E0E7
:1044700088E692E00E94704761E070E08AE692E090
:104480000E947047A89563E770E08CE692E00E9476
:10449000704764E670E08EE692E00E94704764E642
:1044A00070E080E792E00E94704760E070E082E791
:1044B00092E00E94704760E070E084E792E00E9422
:1044C000704760E070E086E792E00E947047A89530
:1044D00060E070E088E792E00E94704760E070E082
:1044E0008AE792E00E94704760E070E08CE792E01B
:1044F0000E94704760E070E08EE792E00E94704793
:10450000A8956EEB70E084E492E00E94704768EC3E
:1045100070E086E492E00E94704766E170E088E413
:1045200092E00E94704766E170E08AE492E00E94A7
:10453000704761E070E08CE492E00E947047A895BB
:1045400064E670E08EE492E00E94704764E670E0FA
:1045500080E592E00E94704764E670E082E592E0B8
:104560000E94704760E070E084E592E00E9470472E
:1045700060E070E086E592E00E94704760E070E0E5
:1045800088E592E00E947047A89560E070E08AE5B7
:1045900092E00E94704760E070E08CE592E00E943B
:1045A000704760E070E08EE592E00E94704760E046
:1045B00070E080E692E00E947047A89566EE70E099
:1045C00086E292E00E94704762EC71E088E292E03D
:1045D0000E94704766E170E08AE292E00E947047B4
:1045E00066E170E08CE292E00E94704761E070E06A
:1045F0008EE292E00E947047A89563E770E080E346
:1046000092E00E94704764E670E082E392E00E94CC
:10461000704764E670E084E392E00E94704760E0D7
:1046200070E086E392E00E94704760E070E088E30B
:1046300092E00E94704760E070E08AE392E00E949E
:104640007047A89560E070E08CE392E00E947047AC
:1046500060E070E08EE392E00E94704760E070E0FE
:1046600080E492E00E94704760E070E082E492E0B3
:104670000E947047A89566EE70E088E092E00E9484
:10468000704762EC71E08AE092E00E94704766E158
:1046900070E08CE092E00E94704766E170E08EE08E
:1046A00092E00E94704761E070E080E192E00E9439
:1046B0007047A89563E770E082E192E00E9470473E
:1046C00064E670E084E192E00E94704764E670E086
:1046D00086E192E00E94704760E070E088E192E03D
:1046E0000E94704760E070E08AE192E00E947047AB
:1046F00060E070E08CE192E00E947047A89560E075
:1047000070E08EE192E00E94704760E070E080E22D
:1047100092E00E94704760E070E082E292E00E94C6
:10472000704760E070E084E292E00E947047A895D4
:1047300063EC70E08CEC91E00E94704766E170E001
:1047400080ED91E00E94704761E070E084ED91E0BF
:104750000E9470476FE070E086ED91E00E94704724
:10476000A89564E670E088ED91E00E94704761E0F2
:1047700070E082EE91E00E94704763EC70E084EE9E
:1047800091E00E9470476AE070E086EE91E00E943E
:104790007047A89562EC71E084E791E00E94704751
:1047A00066E170E088E791E00E94704761E070E0A8
:1047B0008AE791E00E9470476EE670E08CE791E036
:1047C0000E947047A89564E670E080E891E00E943E
:1047D000704762E070E088E891E00E94704762EC08
:1047E00071E08AE191E00E94704766E170E08CE13F
:1047F00091E00E94704762E170E08EE191E00E94DA
:104800007047A89564E670E084E291E00E947047EA
:1048100064E670E086E291E00E94704764E070E038
:104820008EE291E00E9470476CE271E084E391E0D7
:104830000E947047A89562EC71E080EC90E00E94C5
:10484000704766E170E082EC90E00E94704766E19C
:1048500070E084EC90E00E94704761E070E086ECCC
:1048600090E00E947047A8956EE670E088EC90E0BA
:104870000E94704764E670E08AEC90E00E94704706
:1048800064E670E08CEC90E00E94704765E070E0B8
:1048900084ED90E00E947047A89562EC71E086E696
:1048A00090E00E94704766E170E08AE690E00E9426
:1048B000704761E070E08CE690E00E9470476EE621
:1048C00070E08EE690E00E947047A89564E670E084
:1048D00082E790E00E94704766E070E08AE790E02F
:1048E0000E94704763EC70E08CEB92E00E9470478E
:1048F000A89508956FE070E080EE92E00E94704706
:104900006FE070E08EED92E00E9470476FE070E023
:104910008CED92E00E94704761E08BED92E00E9486
:10492000634761E08AED92E00C9463478FB9779B0F
:10493000FECF8FB10895CF93A39AAB9AAB9880E046
:10494000F5DFC82F80E0F2DFAB9A6C2F70E0762F96
:104950006627682B687F7F7723E0769567952A9591
:10496000E1F780E090E00E942D4320E030E040E855
:104970005EE30E9493430E94014370937E0660931E
:104980007D06CB01CF910895CF93A79AAF9AAF98A8
:1049900080E0CCDFC82F80E0C9DFAF9A6C2F70E0D9
:1049A000762F6627682B687F7F7723E0769567955B
:1049B0002A95E1F780E090E00E942D4320E030E06E
:1049C00040E85EE30E9493430E9401437093AC066B
:1049D0006093AB06CB01CF91089586E291E090936E
:1049E000F1068093F00680917E068F9380917D067C
:1049F0008F9383E092E09F938F930E946D448DE0AC
:104A00008A95F1F70000809158068F9380915706A0
:104A10008F938DE092E09F938F930E946D449DE071
:104A20009A95F1F7000080919A061F928F9387E183
:104A300092E09F938F930E946D448DE08A95F1F7E9
:104A400000008091E8061F928F9382E292E09F938C
:104A50008F930E946D449DE09A95F1F700008CE2DF
:104A600092E09F938F930E946D448DE08A95F1F7B9
:104A700000008091AC068F938091AB068F9384E306
:104A800092E09F938F930E946D44A8958DB79EB737
:104A900046960FB6F8949EBF0FBE8DBF80918406D8
:104AA000811108C08DE392E09F938F930E946D4423
:104AB0000F900F90A89580918406813041F484E492
:104AC00092E09F938F930E946D440F900F909DE012
:104AD0009A95F1F70000E09185068E2F90E08830DE
:104AE000910508F09DC0FC01EE58FF4F0C94324434
:104AF0008BE492E09F938F930E946D44A8950F9052
:104B00000F90E091DD068E2F90E08830910508F03F
:104B100087C0FC01E658FF4F0C9432448AE592E0CE
:104B200071C08AE692E06EC082EA92E06BC081EBCF
:104B300092E068C080EC92E065C08FEC92E09F93B9
:104B40008F930E946D44A8950F900F9080918B06D3
:104B5000813009F452C008F44DC0823009F450C0CD
:104B600008958FED92E09F938F930E946D44A895D6
:104B70000F900F9080919206813009F43EC0D0F1E1
:104B8000823009F43DC0089580EF92E042C08EEF7C
:104B900092E09F938F930E946D44A8950F900F9081
:104BA0008091E706813049F128F1823049F108957A
:104BB0008FE093E09F938F930E946D44A8950F9090
:104BC0000F908091DC068130C1F0A0F08230C1F0FE
:104BD000089582E293E09F938F930E946D44A8957D
:104BE0000F900F908091D906813039F018F0823003
:104BF00039F0089585E792E005C084E892E002C0AC
:104C000083E992E09F938F930E946D4407C084E3F1
:104C100093E09F938F930E946D44A8950F900F90FF
:104C20000895CF92DF92EF92FF920F931F93CF934D
:104C3000DF9300D000D0CDB7DEB7809184068130FD
:104C400009F034C18091930690919406892BD9F490
:104C50000FE110E024E230E04AE550E064E670E065
:104C600088E090E00E94CD0A24E230E04AE550E07E
:104C700064E670E08FED90E00E94CD0AA895A49ABA
:104C8000AC980E944612CC24C394D12C8091840607
:104C9000813009F00BC1A895A0DE8091DF069091CC
:104CA000E0068A35910549F42FEF8DE399E4215010
:104CB00080409040E1F700C00000A89503E02FE19C
:104CC00030E04FEF5FEF69E170E085E890E00E942F
:104CD0008F198091630080FD81C0A8951C821B8282
:104CE0001A821982BE016F5F7F4FCE0103960E9428
:104CF00095428B819C818431954088F489819A8189
:104D0000883D9E4060F489819A81853C994038F0C5
:104D1000D0929406C09293061092A20613D48B816F
:104D20009C818431954098F589819A818C3D95408C
:104D300070F589819A81853F914048F1D09294061F
:104D4000C09293061092B30680918506811102C02D
:104D50000E94153880918506813011F40E94013B34
:104D600080918506823011F40E94083C809185066E
:104D7000843011F40E940F3D80918506853009F43E
:104D8000ADD480918506863011F40E940D37809154
:104D90004906813019F58B819C81853C9940F0F062
:104DA00089819A818C3D9540C8F489819A81853F9B
:104DB0009140A0F0D0929406C09293060E94161AD9
:104DC00080E00E942E410E94994110929406109218
:104DD00093068FE190E00E94420C23DFACDD0E943D
:104DE000D317A8958FEF91EE24E08150904020409A
:104DF000E1F700C00000C8DDA8950E945E18E090B1
:104E00009A06F12C02E02FE130E04FEF5FEF6EE603
:104E100070E08CE190E00E94080CE090E806F12C34
:104E20002FE130E04FEF5FEF6EE670E080EF90E053
:104E30000E94080C80914906813011F40E942B4297
:104E40000E947C1180918406811120CFA8950E9438
:104E5000631BA8950E94B81AA8950E9446120FE1FC
:104E600010E029E130E04AE550E06EE670E088E0CD
:104E700090E00E94CD0A29E130E04AE550E06EE67C
:104E800070E08FED90E00E94CD0A8091490681305C
:104E900021F40E9426410E94654210925806109209
:104EA00057061092940610929306F0CE0F900F9032
:104EB0000F900F90DF91CF911F910F91FF90EF9086
:104EC000DF90CF900895EF92FF920F931F93CF93AF
:104ED000DF938091A106813009F047C18FE190E016
:104EE0000E94420C0E948B1485E08093A706C5E0C7
:104EF0008091A106813009F038C10E94CF158091C0
:104F0000A7068230D9F48091D2068F5F8093D206B3
:104F10000FE110E02CE330E046EE50E069E670E08F
:104F200081E090E00E94CD0A22E330E043EC50E0C3
:104F300068E270E088E090E00E94CD0A8091A706C8
:104F40008330D9F48091D20681508093D2060FE14C
:104F500010E02CE330E046EE50E069E670E081E0DE
:104F600090E00E94CD0A22E330E043EC50E068E29A
:104F700070E088E090E00E94CD0A8091D2068530F2
:104F800010F01092D2068091D206823081F1B8F4EE
:104F90008823D9F0813009F0C1C078E0E72E76E0AF
:104FA000F72E01E02FE130E04FEF5FEF6CE370E0B0
:104FB00088E090E00E94C20B8EED92E029C0833021
:104FC000B1F1843009F471C0A9C0E1E2EE2EE6E04F
:104FD000FE2E01E02FE130E04FEF5FEF6CE370E079
:104FE0008FE090E00E94C20B80EE92E011C06CEF67
:104FF000E62E65E0F62E01E02FE130E04FEF5FEFA7
:105000006CE370E082E390E00E94C20B8CED92E0D2
:105010000E9455477C0103E02FE130E04FEF5FEF46
:1050200062E870E080E590E00E94080C77C044EEF2
:10503000E42E45E0F42E01E02FE130E04FEF5FEF8A
:105040006CE370E088E290E00E94C20B52EFE52E24
:1050500055E0F52E02E02FE130E04FEF5FEF62E820
:1050600070E088E290E00E94C20B8091A706811157
:1050700019C0D3D83FDC3EEAE32E35E0F32E2FE112
:1050800030E04FEF5FEF62E870E088E290E00E946E
:10509000C20B2FEF89E698E1215080409040E1F764
:1050A00000C00000C093A70639C023EDE22E25E022
:1050B000F22E01E02FE130E04FEF5FEF6CE370E0A4
:1050C0008EE190E00E94C20B8BED92E00E944D4772
:1050D000813079F495ECE92E95E0F92E03E02FE18B
:1050E00030E04FEF5FEF62E870E080E590E00E9413
:1050F000C20B8BED92E00E944D4781110FC080ECF6
:10510000E82E85E0F82E03E02FE130E04FEF5FEF6F
:1051100062E870E080E590E00E94C20BD091A706A3
:10512000D13069F41092A106109294061092930661
:105130008FE190E00E94420CD093840672DD809152
:10514000A706811106C081E08093A1061092E406B3
:1051500013D0C093A7062FE785EB91E02150804044
:105160009040E1F700C00000C3CEDF91CF911F91C6
:105170000F91FF90EF900895BF92CF92DF92EF9240
:10518000FF920F931F93CF93DF938091E4068111D9
:10519000CFC185E08093A706C9E1D0E025E0C22E0B
:1051A000D12C35E0B32E8091E4068111C1C18091EC
:1051B000D206813009F46FC038F0823009F4DDC0C6
:1051C000843009F441C1A4C180EE92E00E945547A9
:1051D0007C0103E02FE130E040E058EF62E870E04E
:1051E00080E590E00E94080C80EE92E00E94554716
:1051F0009093A6068093A5060E94CF158091A706DE
:105200008230A9F48091A5069091A606019690930C
:10521000A6068093A5060FE110E02CE330E046EEF1
:1052200050E069E670E081E090E00E94CD0A809154
:10523000A7068330A9F48091A5069091A606019750
:105240009093A6068093A5060FE110E02CE330E0D2
:1052500046EE50E069E670E081E090E00E94CD0A01
:105260008091A5069091A6064A9720F0D093A606B5
:10527000C093A5068091A5069091A6060A9720F4F2
:10528000D093A606C093A5066091A5067091A606C8
:1052900080EE92E066C08EED92E00E9455477C0160
:1052A00003E02FE130E040E058EF62E870E080E595
:1052B00090E00E94080C8EED92E00E94554790937A
:1052C0008806809387060E94CF158091A7068230BA
:1052D000A9F480918706909188060196909388069C
:1052E000809387060FE110E02CE330E046EE50E0BB
:1052F00069E670E081E090E00E94CD0A8091A70607
:105300008330A9F480918706909188060197909345
:105310008806809387060FE110E02CE330E046EE2C
:1053200050E069E670E081E090E00E94CD0A809153
:105330008706909188064A9720F0D0938806C093FC
:10534000870680918706909188060A9720F4D0936B
:105350008806C093870660918706709188068EED57
:1053600092E00E9470472FE788E391E0215080404F
:105370009040E1F700C00000CBC08CED92E00E94AD
:1053800055477C0103E02FE130E040E058EF62E850
:1053900070E080E590E00E94080C8CED92E00E94A5
:1053A00055479093A4068093A3060E94CF15809141
:1053B000A7068230A9F48091A3069091A4060196D5
:1053C0009093A4068093A3060FE110E02CE330E055
:1053D00046EE50E069E670E081E090E00E94CD0A80
:1053E0008091A7068330A9F48091A3069091A4062A
:1053F00001979093A4068093A3060FE110E02CE39D
:1054000030E046EE50E069E670E081E090E00E9416
:10541000CD0A8091A3069091A4064F9720F0D092D8
:10542000A406C092A3068091A3069091A4060597B6
:1054300020F4D092A406C092A3066091A3067091B6
:10544000A4068CED92E08DCF8BED92E00E944D474B
:1054500080934B060E94CF158091A706823089F475
:1054600080914B068F5F80934B060FE110E02CE399
:1054700030E046EE50E069E670E081E090E00E94A6
:10548000CD0A8091A706833089F480914B06815024
:1054900080934B060FE110E02CE330E046EE50E045
:1054A00069E670E081E090E00E94CD0A80914B06B1
:1054B000823010F010924B0680914B06813079F4C7
:1054C00095ECE92E95E0F92E03E02FE130E040E085
:1054D00058EF62E870E080E590E00E94C20B809196
:1054E0004B0681110FC080ECE82E85E0F82E03E01A
:1054F0002FE130E040E058EF62E870E080E590E0B6
:105500000E94C20B60914B068BED92E00E946347B4
:105510008091A706813049F48093E4068093A10628
:105520008FE190E00E94420CCEDCB092A7063BCE09
:10553000DF91CF911F910F91FF90EF90DF90CF906F
:10554000BF9008959F92AF92BF92CF92DF92EF9259
:10555000FF920F931F93CF93DF938091A206811147
:10556000B1C08FE190E00E94420C0E94FA1385E0E6
:105570008093A7061092A106C0E089E0E82ED1E052
:1055800097E0D92E26E0C22E35E0F32E44E0B42E6B
:1055900053E0A52E62E0962E8091A206811192C062
:1055A0000E94CF158091A706823069F4CF5F0FE18A
:1055B00010E02CE330E046EE50E069E670E081E078
:1055C00090E00E94CD0A8091A706833069F4C15013
:1055D0000FE110E02CE330E046EE50E069E670E0C9
:1055E00081E090E00E94CD0ACA3008F0C0E08C2F24
:1055F0000E94FB128C2F90E08A309105A0F5FC01EF
:10560000EE57FF4F0C9432441092A106109285067B
:105610002AC01092A106D093850625C01092A1063B
:105620009092850620C01092A106A09285061BC00C
:105630001092A106B092850616C01092A106F092B3
:10564000850611C01092A106C09285060CC010926A
:10565000A106D092850607C0D093A10604C010927F
:10566000A106E09285068091A7068130F9F4809129
:10567000A106813049F4109285061092A2068FE1AE
:1056800090E00E94420C1FDCD093A2061092940678
:10569000109293068091850690E090937406809313
:1056A00073068FE190E00E94420CBBDAF092A706ED
:1056B0002FEF80E792E0215080409040E1F700C05A
:1056C00000006ACFDF91CF911F910F91FF90EF9073
:1056D000DF90CF90BF90AF909F900895EF92FF9290
:1056E0000F931F93CF93DF93A8958091B3068111F9
:1056F000F4C08FE190E00E94420C0E943E15809120
:10570000DC0690E090938E0680938D0685E0809372
:10571000A706C1E0D5E08091B3068111DEC0A8954F
:105720000E94CF158091A7068230A9F480918D0642
:1057300090918E06019690938E0680938D060FE1D0
:1057400010E02CE330E046EE50E069E670E081E0E6
:1057500090E00E94CD0A8091A7068330A9F4809141
:105760008D0690918E06019790938E0680938D06FC
:105770000FE110E02CE330E046EE50E069E670E027
:1057800081E090E00E94CD0A80918D0690918E0676
:10579000039720F010928E0610928D0680918D0650
:1057A00090918E068130910589F1D0F0029709F031
:1057B00046C086E8E82E85E0F82E02E02FE130E0D2
:1057C0004FEF5FEF6DE770E088E290E00E94C20B60
:1057D00082E08093DC064EE150E062E870E02BC08E
:1057E0002AE9E22E25E0F22E02E02FE130E04FEF31
:1057F0005FEF6DE770E088E290E00E94C20B1092CC
:10580000DC064EE150E06EEB70E015C090E9E92E49
:1058100095E0F92E02E02FE130E04FEF5FEF6DE70A
:1058200070E088E290E00E94C20BC093DC064EE17B
:1058300050E060EA70E08DE596E00E943D4780917F
:10584000A70681110FC0A895C093B30610929406C5
:1058500010929306C093A2068FE190E00E94420C42
:10586000A895DFD98091A706813059F5A895809336
:10587000B30610929406109293068093A2068FE1CD
:1058800090E00E94420CA8951092E9068091DC06F7
:10589000813069F038F0823091F44EE150E062E8F6
:1058A00070E009C04EE150E06EEB70E004C04EE1E4
:1058B00050E060EA70E08DE596E00E943D47A895D3
:1058C00013D0D093A7062FEF80E792E021508040BD
:1058D0009040E1F700C000001ECFDF91CF911F91F3
:1058E0000F91FF90EF900895EF92FF920F931F9307
:1058F000CF938091E90681110C9407378FE190E0F6
:105900000E94420C0E94391685E08093A706C5E0EC
:105910008091E90681110C9407370E94CF15809180
:10592000A7068230D9F48091D8068F5F8093D8067D
:105930000FE110E02CE330E046EE50E069E670E065
:1059400081E090E00E94CD0A22E330E043EC50E099
:1059500068E270E088E090E00E94CD0A8091A7069E
:105960008330D9F48091D80681508093D8060FE116
:1059700010E02CE330E046EE50E069E670E081E0B4
:1059800090E00E94CD0A22E330E043EC50E068E270
:1059900070E088E090E00E94CD0A8091D8068E30B9
:1059A00010F01092D806E091D8068E2F90E08E303D
:1059B000910510F00C94C235FC01E457FF4F809123
:1059C00085060C943244811137C080915D06909118
:1059D0005E06893E934020F010925E0610925D06AE
:1059E00078E3E72E75E0F72E01E02FE130E04FEF8E
:1059F0005FEF62E370E08FE090E00E94C20BE1E3B2
:105A0000EE2EE5E0FE2E2FE130E04FEF5FEF66E493
:105A100070E08CE390E00E94C20BE0905D06F09095
:105A20005E0603E02FE130E04FEF5FEF62E870E0E9
:105A300080E590E00E94080C80918506813009F095
:105A4000B6C780915D0690915E06893E934020F036
:105A500010925E0610925D0658E3E52E55E0F52E95
:105A600001E02FE130E04FEF5FEF62E370E08FE0A5
:105A700090E00E94C20B61E3E62E65E0F62E2FE176
:105A800030E04FEF5FEF66E470E08CE390E00E945F
:105A9000C20BE0905D06F0905E067EC7811137C0B4
:105AA00080915F0690916006893E934020F01092AD
:105AB000600610925F0639E1E32E35E0F32E01E037
:105AC0002FE130E04FEF5FEF62E370E08FE090E0B6
:105AD0000E94C20B4BE0E42E45E0F42E2FE130E0B3
:105AE0004FEF5FEF66E470E08CE390E00E94C20B42
:105AF000E0905F06F090600603E02FE130E04FEFAA
:105B00005FEF62E870E080E590E00E94080C809111
:105B10008506813031F48091D8068F5F8093D80656
:105B200039C08230B9F580915F0690916006893E58
:105B3000934020F01092600610925F0699E1E92EE2
:105B400095E0F92E01E02FE130E04FEF5FEF62E3E7
:105B500070E08FE090E00E94C20B2BE0E22E25E087
:105B6000F22E2FE130E04FEF5FEF66E470E08CE360
:105B700090E00E94C20BE0905F06F090600603E0A8
:105B80002FE130E04FEF5FEF62E870E080E590E0FA
:105B90000E94080C809185068430B9F580915F06DB
:105BA00090916006893E934020F01092600610921A
:105BB0005F0609E1E02E05E0F02E01E02FE130E084
:105BC0004FEF5FEF62E370E08FE090E00E94C20B66
:105BD0008BE0E82E85E0F82E2FE130E04FEF5FEF0D
:105BE00066E470E08CE390E00E94C20BE0905F06F8
:105BF000F090600603E02FE130E04FEF5FEF62E8E6
:105C000070E080E590E00E94080C80918506853068
:105C1000B9F580915F0690916006893E934020F02F
:105C20001092600610925F06B9E1EB2EB5E0FB2EF4
:105C300001E02FE130E04FEF5FEF62E370E08FE0D3
:105C400090E00E94C20B1BE0E12E15E0F12E2FE147
:105C500030E04FEF5FEF66E470E08CE390E00E948D
:105C6000C20BE0905F06F090600603E02FE130E0A9
:105C70004FEF5FEF62E870E080E590E00E94080C73
:105C800080918506863009F07DC780915F069091EE
:105C90006006893E934020F01092600610925F06E5
:105CA000F9E1EF2EF5E0FF2E01E02FE130E04FEFBC
:105CB0005FEF62E370E08FE090E00E94C20BABE028
:105CC000EA2EA5E0FA2E2FE130E04FEF5FEF66E419
:105CD00070E08CE390E00E94C20BE0905F06F090D1
:105CE0006006B2C5811136C080916106909162064E
:105CF0004F9720F0109262061092610673EFE72E24
:105D000074E0F72E01E02FE130E04FEF5FEF62E348
:105D100070E08FE090E00E94C20BEBEDEE2EE4E02D
:105D2000FE2E2FE130E04FEF5FEF66E470E08FE092
:105D300090E00E94C20BE0906106F090620603E0E2
:105D40002FE130E04FEF5FEF62E870E080E590E038
:105D50000E94080C80918506813009F028C6809148
:105D60006106909162064F9720F0109262061092A1
:105D7000610653EFE52E54E0F52E01E02FE130E00F
:105D80004FEF5FEF62E370E08FE090E00E94C20BA4
:105D90006BEDE62E64E0F62E2FE130E04FEF5FEF83
:105DA00066E470E08FE090E00E94C20BE090610634
:105DB000F0906206F1C5811136C080916306909122
:105DC00064064F9720F0109264061092630633EC3D
:105DD000E32E34E0F32E01E02FE130E04FEF5FEFF0
:105DE00062E370E08FE090E00E94C20B4BEAE42E89
:105DF00044E0F42E2FE130E04FEF5FEF66E470E017
:105E00008FE090E00E94C20BE0906306F090640681
:105E100003E02FE130E04FEF5FEF62E870E080E5F4
:105E200090E00E94080C80918506813031F48091C9
:105E3000D8068F5F8093D80638C08230B1F5809144
:105E40006306909164064F9720F0109264061092BA
:105E5000630693ECE92E94E0F92E01E02FE130E0A7
:105E60004FEF5FEF62E370E08FE090E00E94C20BC3
:105E70002BEAE22E24E0F22E2FE130E04FEF5FEF2D
:105E800066E470E08FE090E00E94C20BE090630651
:105E9000F090640603E02FE130E04FEF5FEF62E83F
:105EA00070E080E590E00E94080C809185068430C7
:105EB000B1F580916306909164064F9720F010929F
:105EC00064061092630603ECE02E04E0F02E01E07D
:105ED0002FE130E04FEF5FEF62E370E08FE090E0A2
:105EE0000E94C20B8BEAE82E84E0F82E2FE130E00E
:105EF0004FEF5FEF66E470E08FE090E00E94C20B2E
:105F0000E0906306F090640603E02FE130E04FEF8D
:105F10005FEF62E870E080E590E00E94080C8091FD
:105F200085068530B1F580916306909164064F97A0
:105F300020F01092640610926306B3ECEB2EB4E0EE
:105F4000FB2E01E02FE130E04FEF5FEF62E370E006
:105F50008FE090E00E94C20B1BEAE12E14E0F12ECC
:105F60002FE130E04FEF5FEF66E470E08FE090E00C
:105F70000E94C20BE0906306F090640603E02FE1FC
:105F800030E04FEF5FEF62E870E080E590E00E9464
:105F9000080C80918506863009F0F4C5809163066F
:105FA000909164064F9720F0109264061092630659
:105FB000F3ECEF2EF4E0FF2E01E02FE130E04FEFA5
:105FC0005FEF62E370E08FE090E00E94C20BABEA0B
:105FD000EA2EA4E0FA2E2FE130E04FEF5FEF66E407
:105FE00070E08FE090E00E94C20BE0906306F090BA
:105FF00064062AC4811145C08091650690916606A9
:10600000039730F081E090E09093660680936506F8
:10601000E3E9EE2EE4E0FE2E01E02FE130E04FEF69
:106020005FEF6CE370E08FE090E00E94C20B809124
:10603000650690916606019779F475ECE72E75E098
:10604000F72E03E02FE130E04FEF5FEF62E870E002
:1060500080E590E00E94C20B8091650690916606F3
:10606000892B79F460ECE62E65E0F62E03E02FE153
:1060700030E04FEF5FEF62E870E080E590E00E9473
:10608000C20B80918506813009F045C0809165067C
:1060900090916606039730F081E090E09093660659
:1060A0008093650653E9E52E54E0F52E01E02FE1DB
:1060B00030E04FEF5FEF6CE370E08FE090E00E9424
:1060C000C20B8091650690916606019779F445ECC4
:1060D000E42E45E0F42E03E02FE130E04FEF5FEFD8
:1060E00062E870E080E590E00E94C20B8091650656
:1060F00090916606892B79F430ECE32E35E0F32E8F
:1061000003E02FE130E04FEF5FEF62E870E080E501
:1061100090E00E94C20B80918506823009F045C054
:106120008091650690916606039730F081E090E0DB
:10613000909366068093650623E9E22E24E0F22E12
:1061400001E02FE130E04FEF5FEF6CE370E08FE0B4
:1061500090E00E94C20B80916506909166060197BF
:1061600079F495ECE92E95E0F92E03E02FE130E08B
:106170004FEF5FEF62E870E080E590E00E94C20BB5
:106180008091650690916606892B79F480ECE82E63
:1061900085E0F82E03E02FE130E04FEF5FEF62E89B
:1061A00070E080E590E00E94C20B809185069CEF34
:1061B000980F923008F4A5C4863009F0E3C48091AA
:1061C000650690916606039730F081E090E0909329
:1061D00066068093650603E9E02E04E0F02E01E0F8
:1061E0002FE130E04FEF5FEF6CE370E08FE090E085
:1061F0000E94C20B8091650690916606019779F422
:1062000015ECE12E15E0F12E03E02FE130E04FEF29
:106210005FEF62E870E080E590E00E94C20B809141
:10622000650690916606892B09F0ACC4B0ECEB2EA4
:10623000B5E0FB2E03E02FE130E04FEF5FEF62E8C7
:1062400070E080E590E00E94C20B9CC4811137C0D1
:1062500080916706909168068F35914020F01092EA
:10626000680610926706FBE7EF2EF4E0FF2E01E0D0
:106270002FE130E04FEF5FEF62E370E08FE090E0FE
:106280000E94C20BA3E6EA2EA4E0FA2E2FE130E032
:106290004FEF5FEF66E470E08FE090E00E94C20B8A
:1062A000E0906706F090680603E02FE130E04FEFE2
:1062B0005FEF62E870E080E590E00E94080C80915A
:1062C00085068130B9F580916706909168068F3513
:1062D000914020F010926806109267067BE7E72E47
:1062E00074E0F72E01E02FE130E04FEF5FEF62E363
:1062F00070E08FE090E00E94C20BE3E6EE2EE4E057
:10630000FE2E2FE130E04FEF5FEF66E470E08FE0AC
:1063100090E00E94C20BE0906706F090680603E0F0
:106320002FE130E04FEF5FEF62E870E080E590E052
:106330000E94080C809185068230B9F5809167062D
:10634000909168068F35914020F010926806109267
:1063500067065BE7E52E54E0F52E01E02FE130E023
:106360004FEF5FEF62E370E08FE090E00E94C20BBE
:1063700063E6E62E64E0F62E2FE130E04FEF5FEFAC
:1063800066E470E08FE090E00E94C20BE090670648
:10639000F090680603E02FE130E04FEF5FEF62E836
:1063A00070E080E590E00E94080C809185069CEFEB
:1063B000980F923008F4A5C3863009F0E3C38091AA
:1063C0006706909168068F35914020F0109268061C
:1063D000109267063BE7E32E34E0F32E01E02FE155
:1063E00030E04FEF5FEF62E370E08FE090E00E94FB
:1063F000C20B43E6E42E44E0F42E2FE130E04FEFF1
:106400005FEF66E470E08FE090E00E94C20BE090E6
:106410006706F090680618C2811137C0809169063E
:1064200090916A068636910520F010926A061092C5
:1064300069069BE4E92E94E0F92E01E02FE130E0BB
:106440004FEF5FEF62E370E08FE090E00E94C20BDD
:1064500023E3E22E24E0F22E2FE130E04FEF5FEF56
:1064600066E470E08FE090E00E94C20BE090690665
:10647000F0906A0603E02FE130E04FEF5FEF62E853
:1064800070E080E590E00E94080C809185068130E4
:10649000B9F58091690690916A068636910520F0DB
:1064A00010926A06109269060BE4E02E04E0F02ECA
:1064B00001E02FE130E04FEF5FEF62E370E08FE04B
:1064C00090E00E94C20B83E3E82E84E0F82E2FE1D7
:1064D00030E04FEF5FEF66E470E08FE090E00E9405
:1064E000C20BE0906906F0906A0603E02FE130E00D
:1064F0004FEF5FEF62E870E080E590E00E94080CEB
:1065000080918506823031F48091D8068F5F809328
:10651000D80639C08430B9F58091690690916A0631
:106520008636910520F010926A0610926906BBE447
:10653000EB2EB4E0FB2E01E02FE130E04FEF5FEFF8
:1065400062E370E08FE090E00E94C20B13E3E12E63
:1065500014E0F12E2FE130E04FEF5FEF66E470E0E2
:106560008FE090E00E94C20BE0906906F0906A060E
:1065700003E02FE130E04FEF5FEF62E870E080E58D
:1065800090E00E94080C809185068530B9F58091D5
:10659000690690916A068636910520F010926A0687
:1065A00010926906FBE4EF2EF4E0FF2E01E02FE1EC
:1065B00030E04FEF5FEF62E370E08FE090E00E9429
:1065C000C20BA3E3EA2EA4E0FA2E2FE130E04FEF56
:1065D0005FEF66E470E08FE090E00E94C20BE09015
:1065E0006906F0906A0603E02FE130E04FEF5FEFBD
:1065F00062E870E080E590E00E94080C80918506DA
:106600007DC2811137C080916B0690916C068636F1
:10661000910520F010926C0610926B067BE1E72E3C
:1066200074E0F72E01E02FE130E04FEF5FEF62E31F
:1066300070E08FE090E00E94C20BE3E0EE2EE4E019
:10664000FE2E2FE130E04FEF5FEF66E470E08FE069
:1066500090E00E94C20BE0906B06F0906C0603E0A5
:106660002FE130E04FEF5FEF62E870E080E590E00F
:106670000E94080C80918506813031F48091D80603
:106680008F5F8093D80639C08230B9F580916B0650
:1066900090916C068636910520F010926C0610924F
:1066A0006B065BE1E52E54E0F52E01E02FE130E0D2
:1066B0004FEF5FEF62E370E08FE090E00E94C20B6B
:1066C00063E0E62E64E0F62E2FE130E04FEF5FEF5F
:1066D00066E470E08FE090E00E94C20BE0906B06F1
:1066E000F0906C0603E02FE130E04FEF5FEF62E8DF
:1066F00070E080E590E00E94080C8091850684306F
:10670000B9F580916B0690916C068636910520F064
:1067100010926C0610926B063BE1E32E34E0F32EF0
:1067200001E02FE130E04FEF5FEF62E370E08FE0D8
:1067300090E00E94C20B43E0E42E44E0F42E2FE1EF
:1067400030E04FEF5FEF66E470E08FE090E00E9492
:10675000C20BE0906B06F0906C0603E02FE130E096
:106760004FEF5FEF62E870E080E590E00E94080C78
:10677000809185068530B9F580916B0690916C0605
:106780008636910520F010926C0610926B069BE104
:10679000E92E94E0F92E01E02FE130E04FEF5FEFBA
:1067A00062E370E08FE090E00E94C20B23E0E22EF3
:1067B00024E0F22E2FE130E04FEF5FEF66E470E06F
:1067C0008FE090E00E94C20BE0906B06F0906C06A8
:1067D00003E02FE130E04FEF5FEF62E870E080E52B
:1067E00090E00E94080C80918506863009F0CAC1AD
:1067F00080916B0690916C068636910520F0109280
:106800006C0610926B061BE1E12E14E0F12E01E004
:106810002FE130E04FEF5FEF62E370E08FE090E058
:106820000E94C20B83E0E82E84E0F82E2FE130E0D6
:106830004FEF5FEF66E470E08FE090E00E94C20BE4
:10684000E0906B06F0906C0603E02FE130E04FEF34
:106850005FEF62E870E080E590E00E94080C92C172
:10686000811129C080917506909176068D329140F4
:1068700020F01092760610927506B3E8EB2EB3E086
:10688000FB2E01E02FE130E04FEF5FEF6CE370E0B3
:106890008FE090E00E94C20BE0907506F0907606C3
:1068A00003E02FE130E04FEF5FEF62E870E080E55A
:1068B00090E00E94080C80918506813009F077C035
:1068C00080917506909176068D32914020F010925D
:1068D000760610927506A3E8EA2EA3E0FA2E01E0F0
:1068E0002FE130E04FEF5FEF6CE370E08FE090E07E
:1068F0000E94C20BE0907506F09076064DC08111A3
:1069000029C08091770690917806893E934020F0C7
:106910001092780610927706F9EDEF2EF3E0FF2E35
:1069200001E02FE130E04FEF5FEF6CE370E08FE0CC
:1069300090E00E94C20BE0907706F090780603E0AA
:106940002FE130E04FEF5FEF62E870E080E590E02C
:106950000E94080C80918506813049F58091770668
:1069600090917806893E934020F01092780610921C
:106970007706E9EDEE2EE3E0FE2E01E02FE130E0B8
:106980004FEF5FEF6CE370E08FE090E00E94C20B8E
:10699000E0907706F090780603E02FE130E04FEFCB
:1069A0005FEF62E870E080E590E00E94080C809163
:1069B0008506823009F4A5C09CEF980F923008F04C
:1069C0009DC09FC0811190C080916D0690916E0610
:1069D000039720F010926E0610926D0671EFE72E6D
:1069E00073E0F72E01E02FE130E04FEF5FEF6CE353
:1069F00070E08EE190E00E94C20B80916D06909154
:106A00006E06019779F465ECE62E65E0F62E03E05C
:106A10002FE130E04FEF5FEF62E870E080E590E05B
:106A20000E94C20B80916D0690916E06892B79F4BD
:106A300050ECE52E55E0F52E03E02FE130E04FEF6E
:106A40005FEF62E870E080E590E00E94C20B809109
:106A50006D0680934A0648C0811146C080914A065F
:106A6000811108C08DC081113FC080914A068111FB
:106A70009EC186C0813009F085C080916F069091DB
:106A80007006893E934020F01092700610926F06B7
:106A90003BE7E32E34E0F32E01E02FE130E04FEF4F
:106AA0005FEF62E370E08FE090E00E94C20B43EC86
:106AB000E42E43E0F42E2FE130E04FEF5FEF66E489
:106AC00070E08FE090E00E94C20BE0906F06F090C3
:106AD000700603E02FE130E04FEF5FEF62E870E017
:106AE00080E590E00E94080C80918506813049F095
:106AF000823039F0843029F0853019F0863009F081
:106B000041C08091D8068F5F8093D8063BC0882310
:106B100021F09FEF980F923018F41092D8062BC0F6
:106B2000843049F58091790690917A06893E9340A8
:106B300020F010927A06109279068CE5E82E83E018
:106B4000F82E01E02FE130E04FEF5FEF6CE370E0F3
:106B50008FE090E00E94C20BE0907906F0907A06F8
:106B600003E02FE130E04FEF5FEF62E870E080E597
:106B700090E00E94080C809185068550823010F4C8
:106B80001092D8068091A706813009F0F3C0809357
:106B9000E9061092B30680918506811128C0E09124
:106BA0008D06F0918E06E830F10508F5E656FF4FA8
:106BB0004EE150E00C9432446CEB72E014C06EE98C
:106BC00072E011C060E872E00EC062E672E00BC0D5
:106BD00064E472E008C066E272E005C068E072E05A
:106BE00002C06AEE71E08DE596E00E945A478091FE
:106BF00085068130E1F480918D0690918E0681307A
:106C0000910569F038F0029791F44EE150E060E9A7
:106C100071E009C04EE150E06CEC71E004C04EE15F
:106C200050E06EEA71E08DE596E00E945A4780914F
:106C300085068230E1F480918D0690918E06813038
:106C4000910569F038F0029791F44EE150E066E367
:106C500071E009C04EE150E062E771E004C04EE12E
:106C600050E064E571E08DE596E00E945A4780911E
:106C700085068430E1F480918D0690918E068130F6
:106C8000910569F038F0029791F44EE150E06CED17
:106C900070E009C04EE150E068E171E004C04EE1EF
:106CA00050E06AEF70E08DE596E00E945A478091CF
:106CB00085068530E1F480918D0690918E068130B5
:106CC000910569F038F0029791F44EE150E062E8E6
:106CD00070E009C04EE150E06EEB70E004C04EE1A0
:106CE00050E060EA70E08DE596E00E945A4780919E
:106CF00085068630E1F480918D0690918E06813074
:106D0000910569F038F0029791F44EE150E068E2A5
:106D100070E009C04EE150E064E670E004C04EE16E
:106D200050E066E470E08DE596E00E945A478FE1FE
:106D300090E00E94420C80918506811101C075D1BE
:106D400080918506813009F45CD48091850682307B
:106D500009F45ED580918506843009F460D680916F
:106D60008506853011F40E946E2B80918506863051
:106D700009F453D08091A70681110CC081E0809363
:106D8000E9061092B30610927B068FE190E00E9414
:106D9000420CEED2C093A7068FE798E321E0815022
:106DA00090402040E1F700C000000C94882C813016
:106DB00009F0E8CE8091710690917206893E934069
:106DC00020F010927206109271069CEAE92E93E070
:106DD000F92E01E02FE130E04FEF5FEF62E370E06A
:106DE0008FE090E00E94C20B29E9E22E23E0F22E10
:106DF0002FE130E04FEF5FEF66E470E08FE090E06E
:106E00000E94C20BE0907106F090720662CECF91A4
:106E10001F910F91FF90EF900895EF92FF920F93C3
:106E20001F93CF93DF93A8958091B3068111F6C08D
:106E30008FE190E00E94420C0E943E158091D9069D
:106E400090E090938E0680938D0685E08093A70650
:106E5000C1E0D5E08091B3068111E0C0A8950E9401
:106E6000CF158091A7068230A9F480918D0690916C
:106E70008E06019690938E0680938D060FE110E0AA
:106E80002CE330E046EE50E069E670E081E090E00F
:106E90000E94CD0A8091A7068330A9F480918D06C7
:106EA00090918E06019790938E0680938D060FE148
:106EB00010E02CE330E046EE50E069E670E081E05F
:106EC00090E00E94CD0A80918D0690918E060397E6
:106ED00020F010928E0610928D0680918D06909172
:106EE0008E068130910589F1D0F0029709F046C0F5
:106EF00086E8E82E85E0F82E02E02FE130E04FEF43
:106F00005FEF6DE770E088E290E00E94C20B82E0E4
:106F10008093D9064EE150E068E270E02BC02AE988
:106F2000E22E25E0F22E02E02FE130E04FEF5FEF9E
:106F30006DE770E088E290E00E94C20B1092D906E3
:106F40004EE150E064E670E015C090E9E92E95E06E
:106F5000F92E02E02FE130E04FEF5FEF6DE770E0D8
:106F600088E290E00E94C20BC093D9064EE150E047
:106F700066E470E08DE596E00E943D478091A706AB
:106F8000811110C0A895C093B30610929406109278
:106F90009306C093A2068FE190E00E94420CA89550
:106FA0000E9411268091A706813061F5A8958093F3
:106FB000B30610929406109293068093A2068FE176
:106FC00090E00E94420CA8951092E9068091D906A3
:106FD000813069F038F0823091F44EE150E068E29F
:106FE00070E009C04EE150E064E670E004C04EE19C
:106FF00050E066E470E08DE596E00E943D47A8957C
:107000000E94742CD093A7062FEF80E792E02150C6
:1070100080409040E1F700C000001CCFDF91CF918D
:107020001F910F91FF90EF900895AF92BF92CF9272
:10703000DF92EF92FF920F931F93CF93DF93A89568
:107040008091B306811189C18FE190E00E94420CCA
:107050000E943E158091DD0690E090938E0680930D
:107060008D0685E08093A706E7E0DE2EF6E0CF2EC2
:10707000D5E0A4E0BA2EB3E0AB2EC1E08091B30618
:1070800081116BC1A8950E94CF158091A70682300F
:10709000A9F480918D0690918E06019690938E06AC
:1070A00080938D060FE110E02CE330E046EE50E0D7
:1070B00069E670E081E090E00E94CD0A8091A70629
:1070C0008330A9F480918D0690918E06019790935C
:1070D0008E0680938D060FE110E02CE330E046EE43
:1070E00050E069E670E081E090E00E94CD0A809176
:1070F0008D0690918E06089720F010928E061092C1
:107100008D06E0918D06F0918E06E830F10508F0CD
:10711000BEC0EE55FF4F0C94324479EAE72E75E07D
:10712000F72E02E02FE130E04FEF5FEF6DE770E008
:1071300082E390E00E94C20B1092DD064EE150E027
:107140006CEB72E09AC064EAE62E65E0F62E02E08F
:107150002FE130E04FEF5FEF6DE770E082E390E00A
:107160000E94C20BC093DD064EE150E06EE972E072
:1071700084C05AE9E52E55E0F52E02E02FE130E01B
:107180004FEF5FEF6DE770E088E290E00E94C20B86
:1071900082E08093DD064EE150E060E872E06DC071
:1071A00040E9E42E45E0F42E02E02FE130E04FEF1D
:1071B0005FEF6DE770E088E290E00E94C20BA09262
:1071C000DD064EE150E062E672E057C036E8E32E9D
:1071D00035E0F32E02E02FE130E04FEF5FEF6DE797
:1071E00070E088E290E00E94C20BB092DD0644E1BC
:1071F00050E064E472E041C02CE7E22E25E0F22E7C
:1072000002E02FE130E04FEF5FEF6DE770E088E2E2
:1072100090E00E94C20BD093DD064EE150E066E2A2
:1072200072E02BC092E7E92E95E0F92E02E02FE103
:1072300030E04FEF5FEF6DE770E088E290E00E9492
:10724000C20BC092DD064EE150E068E072E015C06E
:1072500088E6E82E85E0F82E02E02FE130E04FEFDF
:107260005FEF6DE770E088E290E00E94C20BD09281
:10727000DD064EE150E06AEE71E08DE596E00E9499
:107280003D478FE59AEE0197F1F700C0000080912D
:10729000A70681110FC0A895C093B306109294065B
:1072A00010929306C093A2068FE190E00E94420CD8
:1072B0000E9411268091A706813009F041C0A8954F
:1072C0008093B30610929406109293068093A206C0
:1072D0008FE190E00E94420C1092E906E091DD06F9
:1072E0008E2F90E08830910540F5FC01E655FF4F68
:1072F0004EE150E00C9432446CEB72E014C06EE945
:1073000072E011C060E872E00EC062E672E00BC08D
:1073100064E472E008C066E272E005C068E072E012
:1073200002C06AEE71E08DE596E00E943D478FE570
:107330009AEE0197F1F700C00000A8950E94742C06
:10734000D093A706A8959FEF20E782E091502040B8
:107350008040E1F700C0000091CEDF91CF911F91F6
:107360000F91FF90EF90DF90CF90BF90AF90089576
:10737000CF93C1E080917B06811141C1E091D80695
:107380008E2F90E08E30910508F030C1FC01EE5454
:10739000FF4F0C94324460915D0670915E067093CD
:1073A0004F0660934E068EE591E00E943708909359
:1073B0004F0680934E0690935E0680935D060DC146
:1073C00060915F067091600670939F0660939E06C1
:1073D00082EC91E00E94370890939F0680939E066E
:1073E0009093600680935F06F8C06091610670918B
:1073F00062066093E506772789E190E00E943708EE
:107400008093E50699279093620680936106E5C014
:10741000609163067091640660938A06772789E11C
:1074200090E00E94370880938A069927909364061B
:1074300080936306D2C0809165068093B2060E9455
:1074400046098093B20690E09093660680936506A5
:10745000C4C06091670670916806609389067727BB
:1074600088EC90E00E9437088093890699279093D2
:10747000680680936706B1C06091690670916A06DC
:1074800060939806772784E690E00E9437088093FF
:107490009806992790936A06809369069EC060912A
:1074A0006B0670916C0660939706772784E690E0F0
:1074B0000E94370880939706992790936C068093D3
:1074C0006B068BC060917506709176067093D4063A
:1074D0006093D30688EC90E00E9437089093D4061E
:1074E0008093D306909376068093750676C060915C
:1074F00077067091780670935C0660935B0684E66D
:1075000090E00E94370890935C0680935B0690930E
:1075100078068093770661C080916D0680934A0655
:107520000E944609823018F480934A0602C01092E5
:107530004A0680914A0690E090936E0680936D060D
:107540004CC080914A06811103C01092D8064EC0EB
:10755000813009F04BC060916F0670917006709396
:10756000D6066093D5068AEF90E00E943708909384
:10757000D6068093D5069093700680936F062DC033
:1075800080914A06882309F3813081F56091710664
:10759000709172066093B106772786E490E00E94AE
:1075A00037088093B10699279093720680937106ED
:1075B00014C06091790670917A0670938106609389
:1075C000800684E893E00E943708909381068093B8
:1075D000800690937A06809379062FE788E391E0FE
:1075E000215080409040E1F700C00000C0937B062E
:1075F0001092E9060E945D080E94742CBBCECF91C8
:107600000895EF92FF920F931F93CF93DF93A89566
:107610008091B3068111F5C08FE190E00E94420C89
:107620000E943E1580918B0690E090938E06809389
:107630008D0685E08093A706C1E0D5E08091B30672
:107640008111DFC0A8950E94CF158091A7068230D6
:10765000A9F480918D0690918E06019690938E06E6
:1076600080938D060FE110E02CE330E046EE50E011
:1076700069E670E081E090E00E94CD0A8091A70663
:107680008330A9F480918D0690918E060197909396
:107690008E0680938D060FE110E02CE330E046EE7D
:1076A00050E069E670E081E090E00E94CD0A8091B0
:1076B0008D0690918E06039720F010928E06109200
:1076C0008D06A89580918D0690918E06813091054A
:1076D00089F1D0F0029709F046C086E8E82E85E0EF
:1076E000F82E02E02FE130E04FEF5FEF6DE770E042
:1076F00088E290E00E94C20B82E080938B064EE10C
:1077000050E060E971E02BC02AE9E22E25E0F22E7C
:1077100002E02FE130E04FEF5FEF6DE770E088E2CD
:1077200090E00E94C20B10928B064EE150E06CEC90
:1077300071E015C090E9E92E95E0F92E02E02FE105
:1077400030E04FEF5FEF6DE770E088E290E00E947D
:10775000C20BC0938B064EE150E06EEA71E08DE5FE
:1077600096E00E943D478091A70681110FC0A89521
:10777000C093B3061092940610929306C093A2068B
:107780008FE190E00E94420C0E9411268091A70692
:10779000813059F5A8958093B30610929406109203
:1077A00093068093A2068FE190E00E94420C109213
:1077B000E90680918B06813069F038F0823091F4CF
:1077C0004EE150E060E971E009C04EE150E06CEC40
:1077D00071E004C04EE150E06EEA71E08DE596E0A4
:1077E0000E943D47A8950E94742CD093A7062FEFC6
:1077F00080E792E0215080409040E1F700C0000017
:107800001DCFDF91CF911F910F91FF90EF900895C1
:10781000EF92FF920F931F93CF93DF93A8958091E0
:10782000B3068111F5C08FE190E00E94420C0E94E6
:107830003E158091920690E090938E0680938D067F
:1078400085E08093A706C1E0D5E08091B306811161
:10785000DFC0A8950E94CF158091A7068230A9F4B9
:1078600080918D0690918E06019690938E0680935E
:107870008D060FE110E02CE330E046EE50E069E6C3
:1078800070E081E090E00E94CD0A8091A7068330ED
:10789000A9F480918D0690918E06019790938E06A3
:1078A00080938D060FE110E02CE330E046EE50E0CF
:1078B00069E670E081E090E00E94CD0A80918D063B
:1078C00090918E06039720F010928E0610928D06EE
:1078D00080918D0690918E068130910589F1D0F0CE
:1078E000029709F046C086E8E82E85E0F82E02E00F
:1078F0002FE130E04FEF5FEF6DE770E088E290E05E
:107900000E94C20B82E0809392064EE150E066E353
:1079100071E02BC02AE9E22E25E0F22E02E02FE1F1
:1079200030E04FEF5FEF6DE770E088E290E00E949B
:10793000C20B109292064EE150E062E771E015C072
:1079400090E9E92E95E0F92E02E02FE130E04FEFCB
:107950005FEF6DE770E088E290E00E94C20BC09399
:1079600092064EE150E064E571E08DE596E00E94FC
:107970003D478091A706811110C0A895C093B3061A
:107980001092940610929306C093A2068FE190E0A5
:107990000E94420CA8950E9411268091A706813072
:1079A00059F5A8958093B306109294061092930609
:1079B0008093A2068FE190E00E94420C1092E906AB
:1079C00080919206813069F038F0823091F44EE176
:1079D00050E066E371E009C04EE150E062E771E01B
:1079E00004C04EE150E064E571E08DE596E00E9450
:1079F0003D47A8950E94742CD093A7062FEF80E7EF
:107A000092E0215080409040E1F700C000001DCF7F
:107A1000DF91CF911F910F91FF90EF900895EF921A
:107A2000FF920F931F93CF93DF93A8958091B30696
:107A30008111F6C08FE190E00E94420C0E943E1539
:107A40008091E70690E090938E0680938D0685E006
:107A50008093A706C1E0D5E08091B3068111E0C014
:107A6000A8950E94CF158091A7068230A9F4809135
:107A70008D0690918E06019690938E0680938D06CA
:107A80000FE110E02CE330E046EE50E069E670E0F4
:107A900081E090E00E94CD0A8091A7068330A9F48E
:107AA00080918D0690918E06019790938E0680931B
:107AB0008D060FE110E02CE330E046EE50E069E681
:107AC00070E081E090E00E94CD0A80918D06909157
:107AD0008E06039720F010928E0610928D068091EC
:107AE0008D0690918E068130910589F1D0F0029734
:107AF00009F046C086E8E82E85E0F82E02E02FE186
:107B000030E04FEF5FEF6DE770E088E290E00E94B9
:107B1000C20B82E08093E7064EE150E06CED70E02E
:107B20002BC02AE9E22E25E0F22E02E02FE130E020
:107B30004FEF5FEF6DE770E088E290E00E94C20BCC
:107B40001092E7064EE150E068E171E015C090E95F
:107B5000E92E95E0F92E02E02FE130E04FEF5FEFE4
:107B60006DE770E088E290E00E94C20BC093E706E8
:107B70004EE150E06AEF70E08DE596E00E943D47EF
:107B80008091A706811110C0A895C093B3061092EA
:107B9000940610929306C093A2068FE190E00E9493
:107BA000420CA8950E9411268091A706813061F5AC
:107BB000A8958093B3061092940610929306809332
:107BC000A2068FE190E00E94420CA8951092E9066F
:107BD0008091E706813069F038F0823091F44EE10F
:107BE00050E06CED70E009C04EE150E068E171E0FA
:107BF00004C04EE150E06AEF70E08DE596E00E942F
:107C00003D47A8950E94742CD093A7062FEF80E7DC
:107C100092E0215080409040E1F700C000001CCF6E
:107C2000DF91CF911F910F91FF90EF9008950F93E7
:107C30001F9380918406811199C08091DF069091F5
:107C4000E0068335910591F581E0809384060E94DA
:107C50004C1B0FE110E02CE330E044E650E06BE415
:107C600070E08EE690E00E94CD0A24E230E04AE522
:107C700050E064E670E088E090E00E94CD0A24E2E3
:107C800030E04AE550E064E670E088E090E00E9471
:107C9000CD0A24E230E04AE550E064E670E08FED82
:107CA00090E00E94CD0A0E941126A8950E94ED2422
:107CB0000E94C220A89503E02FE130E04FEF5FEF74
:107CC00069E170E085E890E00E948F190E949B2492
:107CD0000E944A11809184068130A9F5A8950E94DE
:107CE0004C1B0FE110E02CE330E044E650E06BE485
:107CF00070E08EE690E00E94CD0A24E230E04AE592
:107D000050E064E670E088E090E00E94CD0A24E252
:107D100030E04AE550E064E670E088E090E00E94E0
:107D2000CD0A24E230E04AE550E064E670E08FEDF1
:107D300090E00E94CD0A80914906813009F4D5D1A6
:107D40000E941126A8952FEF81EE94E021508040EB
:107D50009040E1F700C000000E94D3170E94C424A5
:107D60000E945E181F910F910C94D7181F910F91CC
:107D700008951F920F920FB60F9211248F939F9325
:107D80008CB190E09093E0068093DF069F918F91F5
:107D90000F900FBE0F901F9018951F920F920FB665
:107DA0000F9211242F938F939F9380915706909158
:107DB00058060196883E23E0920728F490935806CF
:107DC0008093570604C0109258061092570680916F
:107DD0008206811105C01092E2061092E1060BC0E6
:107DE000813049F48091E1069091E20601969093EA
:107DF000E2068093E10680919C06811105C01092F5
:107E00005606109255060BC0813049F480915506F4
:107E10009091560601969093560680935506809150
:107E20009506811105C010925A06109259060BC092
:107E3000813049F48091590690915A0601969093A9
:107E40005A06809359069F918F912F910F900FBEE4
:107E50000F901F9018958091640088608093640053
:107E6000809165008860809365002FEF89E698E136
:107E7000215080409040E1F700C000008FEF8ABBA6
:107E800081BB80936100C1E0C4BBA89588EA8FBD27
:107E90008CE08EBD1DBC1CBC17BC16BC8AE78BBD1C
:107EA00082E18ABD19BC18BC10927900109278004A
:107EB00080E187BF10BE87E683BF12BE11BE81E896
:107EC00080938B0085E080938A0010928900109245
:107ED000880010928100109280001092870010920A
:107EE00086001092850010928400109283001092F8
:107EF00082001BB888E98AB986E0809395001092C9
:107F000090008FE289B98FE181BD8FE081BDA89596
:107F1000F9D2A89581E00E94D909A8958FE190E057
:107F20000E94420CA895C093840610928506109278
:107F300058061092570610929A0610925406109204
:107F400083061092E30610927C0680E590E0909301
:107F5000E0068093DF06809164008E7F809364004A
:107F600080916500816080936500C0934906A29A64
:107F7000AA9A809164008260809364008091650079
:107F80008260809365007894A49AAC9A2FEF85EA7A
:107F90009EE0215080409040E1F700C00000A8958D
:107FA000AC988AED92E079D7813011F4A8950FC092
:107FB0000E940D21A8950E947A24A89561E08BED7E
:107FC00092E081D7A89561E08AED92E07CD7A895F0
:107FD00080918406813021F4A8950E941126A895ED
:107FE000A89525DEF4CF80916400806180936400C1
:107FF0008091650080618093650080916400886055
:108000008093640080916500877F809365008091F4
:108010004106909142068536910500F580916400F5
:108020008460809364008091650084608093650023
:1080300087EB9BE00197F1F700C00000A8958091C5
:1080400065008B7F80936500809141069091420688
:1080500001969093420680934106D9CF80916500A6
:1080600088608093650008958091640080618093AA
:108070006400809165008F7E80936500809164002C
:1080800088608093640080916500877F809365009D
:1080900080914106909142068536910500F58091C8
:1080A00064008460809364008091650084608093A4
:1080B000650087EB9BE00197F1F700C00000A895F1
:1080C000809165008B7F809365008091410690913F
:1080D000420601969093420680934106D9CF809143
:1080E0006500886080936500089582EE92E0D5D6A1
:1080F0008093EB06A8958091640080618093640072
:108100008091650080618093650080916400886043
:108110008093640080916500877F809365008091E3
:10812000EB0624E6829FC001112420913F06309186
:1081300040062817390700F5809164008460809319
:1081400064008091650084608093650087EB9BE00C
:108150000197F1F700C00000A895809165008B7F22
:108160008093650080913F06909140060196909320
:10817000400680933F06D3CF80916500886080934E
:108180006500109245061092400610923F06A89591
:108190000895AC01A8958091450681114BC090913E
:1081A0006400906190936400909165009F7E90932D
:1081B00065009091640098609093640090916500D0
:1081C000977F9093650084E6849F9001859F300D92
:1081D000112480913F06909140068217930700F585
:1081E0008091640084608093640080916500846065
:1081F0008093650087EB9BE00197F1F700C00000DA
:10820000A895809165008B7F8093650080913F06E3
:108210009091400601969093400680933F06D9CFF7
:1082200080916500886080936500109240061092EE
:108230003F06A895A89581E0809345060895A895E6
:10824000682F82EE92E03FD6A8950895A89582EE19
:1082500092E023D690E09DDFA8950895A89580939D
:1082600044060895CF93DF9300D000D0CDB7DEB79A
:10827000809163001C821B821A821982BE016F5F8B
:108280007F4FCE01039651D18B819C8184319540E3
:1082900068F489819A81843A964040F489819A8170
:1082A0008D32914018F082E08093ED068B819C81A5
:1082B0008937954090F08B819C81843C994068F48B
:1082C00089819A81843A964040F489819A818D32DD
:1082D000914018F083E08093ED068B819C81893278
:1082E0009A4068F089819A8184379E4040F4898160
:1082F0009A81813D974018F081E08093ED068B8153
:108300009C81863F994060F48B819C8181349640AA
:1083100038F089819A81813D974010F01092ED06E6
:108320008091ED060F900F900F900F90DF91CF91FD
:108330000895DF92EF92FF920F931F93CF93DF93F5
:10834000A89585E08093ED06DBE485E0D82E80914A
:108350004406811178C0A89585DFE0904306F12C92
:1083600003E02FE130E040E058EF62E870E080E5A4
:1083700090E00E94080C8091ED068330C1F4A8952E
:1083800080914306815080934306109242061092DA
:1083900041060FE110E02CE330E046EE50E069E6E4
:1083A00070E081E090E00E94CD0A1DDEA8958091EA
:1083B000ED068230D1F4A895809143068B34A8F461
:1083C000A8958F5F80934306109242061092410653
:1083D0000FE110E02CE330E046EE50E069E670E09B
:1083E00081E090E00E94CD0A3FDE809143068C340C
:1083F00010F0D09343068091ED0681110EC00FE17D
:1084000010E02CE330E046EE50E069E670E081E0F9
:1084100090E00E94CD0A10924306C091ED06C13053
:1084200079F4A895809143060ADFA89580914306C8
:1084300090E05BDEA89510924306A895C093440691
:10844000D092ED0684CFDF91CF911F910F91FF90D5
:10845000EF90DF900895EF92FF920F931F93A895EE
:1084600082EE92E01AD58C3418F48093EC0614C096
:10847000A8951092EC0660E082EE92E024D50FE120
:1084800010E028E230E048E550E06FEA70E080EE6E
:1084900090E00E94CD0AA8958091EC06882381F097
:1084A00082EE92E0FAD4E82EF12C02E02FE130E0E7
:1084B0004FEF5FEF6AEA70E080EF90E00E94080CF7
:1084C0001F910F91FF90EF900895EF92FF920F93FD
:1084D000E090EC06F12C02E02FE130E04FEF5FEF8F
:1084E0006AEA70E080EF90E00E94080C0F91FF9024
:1084F000EF900895C098AB9AAF9A8FB9779BFECF53
:108500008FB1089587E087BBC09AAB9AAF9A83E595
:108510008DB91EB880E8EEDF80E0ECDF80E0EADFB6
:108520008AE18A95F1F700C00895EF92FF920F93C8
:108530001F93CF93DF9300D000D0CDB7DEB77C017F
:108540008B01A895AB9AAF9A1C821B821A82198262
:1085500080EDD0DF80E0CEDF8FB190E09C838B8315
:108560008B819C81982F88279C838B8380E0C2DF3E
:108570002FB18B819C81822B9C838B838B819C81EF
:1085800033E0969587953A95E1F79C838B8387EC4A
:1085900090E00197F1F700C0000080E9ABDF80E0D8
:1085A000A9DF8FB190E09A83898389819A81982F7E
:1085B00088279A83898380E09DDF2FB189819A8102
:1085C000822B9A83898389819A8153E09695879536
:1085D0005A95E1F79A8389838B819C81F701918376
:1085E000808389819A81F801918380830F900F9015
:1085F0000F900F90DF91CF911F910F91FF90EF900F
:10860000089570D088F09F5790F0B92F9927B751EF
:10861000A0F0D1F0660F771F881F991F1AF0BA9546
:10862000C9F712C0B13081F077D0B1E0089574C0BD
:10863000672F782F8827B85F39F0B93FCCF386953C
:1086400077956795B395D9F73EF490958095709599
:1086500061957F4F8F4F9F4F0895E89409C097FB16
:108660003EF490958095709561957F4F8F4F9F4F09
:108670009923A9F0F92F96E9BB279395F69587954D
:1086800077956795B795F111F8CFFAF4BB0F11F410
:1086900060FF1BC06F5F7F4F8F4F9F4F16C08823B7
:1086A00011F096E911C0772321F09EE8872F762FED
:1086B00005C0662371F096E8862F70E060E02AF02E
:1086C0009A95660F771F881FDAF7880F969587951A
:1086D00097F9089557FD9058440F551F59F05F3F83
:1086E00071F04795880F97FB991F61F09F3F79F0D4
:1086F00087950895121613061406551FF2CF469556
:10870000F1DF08C0161617061806991FF1CF8695D7
:108710007105610508940895E894BB2766277727BB
:10872000CB0197F908950BD078C069D028F06ED0AE
:1087300018F0952309F05AC05FC01124EECFCADFAC
:10874000A0F3959FD1F3950F50E0551F629FF00164
:10875000729FBB27F00DB11D639FAA27F00DB11DBD
:10876000AA1F649F6627B00DA11D661F829F222746
:10877000B00DA11D621F739FB00DA11D621F839FCD
:10878000A00D611D221F749F3327A00D611D231FA3
:10879000849F600D211D822F762F6A2F11249F57F1
:1087A00050408AF0E1F088234AF0EE0FFF1FBB1F14
:1087B000661F771F881F91505040A9F79E3F5105B3
:1087C00070F014C0AACF5F3FECF3983EDCF38695BF
:1087D00077956795B795F795E7959F5FC1F7FE2B5E
:1087E000880F911D9695879597F9089597F99F673A
:1087F00080E870E060E008959FEF80EC0895002429
:108800000A941616170618060906089500240A94F5
:1088100012161306140605060895092E0394000C7B
:1088200011F4882352F0BB0F40F4BF2B11F460FF0A
:1088300004C06F5F7F4F8F4F9F4F0895AA1BBB1BD4
:1088400051E107C0AA1FBB1FA617B70710F0A61B50
:10885000B70B881F991F5A95A9F780959095BC0171
:10886000CD010895EE0FFF1F0024001C0BBE0790E2
:10887000F691E02D0994A29FB001B39FC001A39F80
:10888000700D811D1124911DB29F700D811D112449
:10889000911D0895BB274A3031F4992322F4BDE29B
:1088A000909581959F4F01C0BB27FB015527AA27B3
:1088B000880F991FAA1FA41710F0A41B839550516D
:1088C000B9F7A05DAA3308F0A95DA193009779F7E5
:1088D000B111B1931192CB0126C2CF93DF93CDB7E3
:1088E000DEB7AE014B5F5F4FFA0161917191AF014D
:1088F0008091F0069091F10603D0DF91CF91089519
:108900002F923F924F925F926F927F928F929F929F
:10891000AF92BF92CF92DF92EF92FF920F931F938D
:10892000CF93DF93CDB7DEB72B970FB6F894DEBFAA
:108930000FBECDBF6C017B018A01FC01178216823C
:10894000838181FFBFC1CE0101963C01F601938175
:10895000F70193FD859193FF81917F01882309F4AD
:10896000ADC1853239F493FD859193FF81917F01EB
:10897000853221F4B60190E0E6D1E8CF912C212C8C
:10898000312CFFE1F315D8F08B3279F038F48032D6
:1089900079F08332A1F4232D20611DC08D3261F066
:1089A000803369F4232D216016C0832D8260382E18
:1089B000E32DE4603E2E2AC0F32DF8601DC037FC85
:1089C0002DC020ED280F2A3040F08E32B9F436FC4D
:1089D00075C1232D2064322E19C036FE06C08AE0F0
:1089E000989E200D1124922E11C0EAE02E9E200D9B
:1089F0001124222EF32DF0623F2E08C08C3621F474
:108A0000832D8068382E02C0883641F4F70193FD2B
:108A1000859193FF81917F018111B3CF982F9F7D25
:108A20009554933028F40C5F1F4F9FE399830DC03A
:108A3000833631F0833771F0833509F055C020C09B
:108A4000F801808189830E5F1F4F88248394912CC5
:108A5000530112C02801F2E04F0E511CF801A08012
:108A6000B18036FE03C0692D70E002C06FEF7FEF6A
:108A7000C5014ED14C018201F32DFF773F2E15C069
:108A8000280122E0420E511CF801A080B18036FE80
:108A900003C0692D70E002C06FEF7FEFC5012DD1DB
:108AA0004C01F32DF0683F2E820133FC19C0822D5A
:108AB00090E088169906A0F4B60180E290E043D1D8
:108AC0002A94F5CFF50137FC859137FE81915F013E
:108AD000B60190E038D121102A9421E0821A910841
:108AE0008114910479F7E1C0843611F0893639F5A3
:108AF000F80137FE07C060817181828193810C5F2C
:108B00001F4F08C060817181072E000C880B990BE4
:108B10000E5F1F4FF32DFF763F2E97FF09C09095F4
:108B20008095709561957F4F8F4F9F4FF0683F2ED6
:108B30002AE030E0A30143D1882E861844C085374F
:108B400031F4232D2F7EB22E2AE030E025C0932D64
:108B5000997FB92E8F36C1F018F4883579F0AEC000
:108B6000803719F0883721F0A9C0E92FE061BE2EC7
:108B7000B4FE0DC0FB2DF460BF2E09C034FE0AC048
:108B8000292F2660B22E06C028E030E005C020E183
:108B900030E002C020E132E0F801B7FE07C060819A
:108BA0007181828193810C5F1F4F06C0608171814A
:108BB00080E090E00E5F1F4FA30101D1882E861840
:108BC000FB2DFF773F2E36FE0DC0232D2E7FA22ECC
:108BD000891458F434FE0BC032FC09C0832D8E7EFC
:108BE000A82E05C0B82CA32C03C0B82C01C0B92CEA
:108BF000A4FE0FC0FE01E80DF11D8081803321F439
:108C00009A2D997EA92E09C0A2FE06C0B394B394F2
:108C100004C08A2D867809F0B394A3FC10C0A0FE8E
:108C200006C0B21480F4280C922C9B180DC0B2140C
:108C300058F4B60180E290E086D0B394F8CFB21435
:108C400018F42B1802C0982C212CA4FE0FC0B601DA
:108C500080E390E078D0A2FE16C0A1FC03C088E7B4
:108C600090E002C088E590E0B6010CC08A2D8678BD
:108C700051F0A1FE02C08BE201C080E2A7FC8DE2B0
:108C8000B60190E060D0891430F4B60180E390E042
:108C90005AD09A94F8CF8A94F301E80DF11D80819F
:108CA000B60190E050D08110F6CF222009F44ECECC
:108CB000B60180E290E047D02A94F7CFF601868192
:108CC000978102C08FEF9FEF2B960FB6F894DEBF0F
:108CD0000FBECDBFDF91CF911F910F91FF90EF900D
:108CE000DF90CF90BF90AF909F908F907F906F90CC
:108CF0005F904F903F902F900895FC010590615038
:108D000070400110D8F7809590958E0F9F1F0895A1
:108D1000FC016150704001900110D8F7809590954A
:108D20008E0F9F1F0895DC01FC01672F719177233F
:108D3000E1F7329704C07C916D9370836291AE1716
:108D4000BF07C8F308950F931F93CF93DF93FB01E1
:108D5000238121FD03C08FEF9FEF2CC022FF16C09F
:108D600046815781248135814217530744F4A081FD
:108D7000B1819D012F5F3F4F318320838C932681EA
:108D800037812F5F3F4F3783268314C08B01EC015F
:108D9000FB010084F185E02D0995892BE1F6D801CE
:108DA00016968D919C911797019617969C938E938A
:108DB0001697CE01DF91CF911F910F910895FA017F
:108DC000AA27283051F1203181F1E8946F936E7F0A
:108DD0006E5F7F4F8F4F9F4FAF4FB1E03ED0B4E0FB
:108DE0003CD0670F781F891F9A1FA11D680F791F3C
:108DF0008A1F911DA11D6A0F711D811D911DA11D4D
:108E000020D009F468943F912AE0269F112430195C
:108E1000305D3193DEF6CF010895462F4770405DF7
:108E20004193B3E00FD0C9F7F6CF462F4F70405DA6
:108E30004A3318F0495D31FD4052419302D0A9F701
:108E4000EACFB4E0A6959795879577956795BA95FB
:108E5000C9F700976105710508959B01AC010A2EC1
:108E600006945795479537952795BA95C9F7620F98
:108E7000731F841F951FA01D0895DC01CB01FC0109
:108E8000E199FECF06C0FFBBEEBBE09A31960DB272
:108E90000D9241505040B8F70895E199FECF9FBB25
:108EA0008EBBE09A99278DB30895A8E1B0E042E027
:108EB00050E0E5CFDC01CB0102C02D9105D041503F
:108EC0005040D8F70895262FE199FECF9FBB8EBB67
:108ED0002DBB0FB6F894E29AE19A0FBE0196089561
:0A8EE000F2DF272FF1CFF894FFCF47
:108EEA00140048005D0078009600B600D500F30033
:108EFA0010012C01490163017C019401AC01C101FB
:108F0A00D501E801010E00000002000000002A0F4E
:108F1A000000000044656C004F4E004F464600209A
:108F2A0020D1F2E0EDF6E8FF00C2E5F0F5EDE8E960
:108F3A0000CDE8E6EDE8E900D0F3F7EDEEE900D080
:108F4A00E5E1EEEBEBE8EDE32000D1F3F8EAE0002F
:108F5A00ECE8EAF0EEF1F5E5EC00EFEBE0F200CA3E
:108F6A00E0EBE8E1F0EEE2EAE000EDE8E7E000CC71
:108F7A00EEF9EDEEF1F2FC00E2E5F0F5E000C2E513
:108F8A00F0F5EDE8E920EDE0E3F02E00CDE8E6EDBE
:108F9A00E8E920EDE0E3F02E20002020D0F3F7ED01
:108FAA00EEE92020200020D1F3F8EAE020EFEBE000
:108FBA00F22000C4EEEF2E20EDE0F1F2F0EEE9EA45
:108FCA00E8002020D1F2E5EAEBEE00CAE0EBE8E1A6
:108FDA00F0EEE2EAE02000EDE8E7E02000C2DBD5AF
:108FEA00CEC40057543D2025750A47530047533DC8
:108FFA002025750A534E00534E3D2025750A454ECD
:10900A004400574B3D2025750A565000503D332EDB
:10901A00360A5200524C3D2025750A68004F3D73AE
:10902A00740A5300473D73740A530053523D5374F4
:10903A006174696F6E200A57500057503D536E365F
:10904A00332F506233370A57540057503D536E41FD
:10905A00670A57540057503D50726F66696C653005
:10906A000A57540057503D50726F66696C65310A51
:10907A0057540057503D50726F66696C65320A57F3
:10908A00540057503D50726F66696C65330A5754E5
:10909A000057503D50726F66696C65340A57540028
:1090AA0057503D50726F66696C65350A57540053C4
:1090BA00523D5550686561746572200A57500053D5
:1090CA00523D507265686561746572200A57500096
:1090DA0053523D4D616E75616C200A5750005352D0
:1090EA003D5265626F6C6C696E67200A5750005377
:1090FA00523D4368697068656174696E67200A57F2
:10910A00500053523D50434268656174696E67204E
:10911A000A57500053523D5043200A575000C2FB91
:10912A00E1E5F0E8F2E520E2FBF1EEF2F3004D3280
:10913A0043726166742056352E347A00202020C28C
:10914A00F0E5ECFF20F0E5E1EEEBEBE8EDE3E02003
:10915A0020202000C2FBE1E5F0E8F2E520F0E5E698
:10916A00E8EC00D2E5ECEFE5F0E0F2F3F0E020EF16
:10917A00EEEBEEF7EAE8202000EDE8E7E020EFF07A
:10918A00E820E4EEEDE0E3F0E5E2E500D2E5ECEF1D
:10919A00E5F0E0F2F3F0E020F3E2E5EBE8F7E5EDE5
:1091AA00E8FF00202020202020E4EEEDE0E3F0E5B7
:1091BA00E2E020202020202000C4EBE8F2E5EBFCCE
:1091CA00EDEEF1F2FC20E2EFE8F2FBE2E0EDE8FF7F
:1091DA0000D4F3EDEAF6E8FF20E4EEEDEEE3F0E585
:1091EA00E2E000EDE8E6EDE5E3EE20EDE0E3F0E5B0
:1091FA00E2E0F2E5EBFF2020202000CCE0EAF1E8F3
:10920A00ECE0EBFCEDE0FF20ECEEF9EDEEF1F2FC28
:10921A00202000E2E5F0F5EDE5E3EE20EDE0E3F0F5
:10922A00E5E2E0F2E5EBFF20202000CCE0EAF1E8FD
:10923A00ECE0EBFCEDE0FF20ECEEF9EDEEF1F2FCF8
:10924A00202000E2E5F0F5EDE5E3EE20EDE0E3F0C5
:10925A00E5E2E0F2E5EBFF20202000D2E5ECEFE5C5
:10926A00F0E0F2F3F0E020E2EAEBFEF7E5EDE8FFEA
:10927A00202000CAEEEDF2F0EEEBFC20EFEE20E249
:10928A00E5F0F5F320202020202000EDE8E6EDE5CA
:10929A00E3EE20EDE0E3F0E5E2E0F2E5EBFF20208B
:1092AA00202000CAEEFDF4F4E8F6E8E5EDF220EF3E
:1092BA00F0EEF4E8EBFF2020202000E2E5F0F5EDE7
:1092CA00E5E3EE20EDE0E3F0E5E2E0F2E5EBFF2096
:1092DA00202000CAEEFDF4F4E8F6E8E5EDF220EF0E
:1092EA00F0EEF4E8EBFF2020202000EDE0E3F0E5CB
:1092FA00E2E0F2E5EBFF202000D2E5ECEFE5F0E05A
:10930A00F2F3F0E020EDE8E6EDE5E3EE20202020A0
:10931A0000EFE0E9EAE82000D2E5ECEFE5F0E0F260
:10932A00F3F0E020ECE5F1F2E0202020202000C25A
:10933A00FBE1E5F0E8F2E520EFF0EEF4E8EBFC0003
:10934A0036302D393020D100CFF0EEF4E8EBFC2096
:10935A003500CFF0EEF4E8EBFC203400CFF0EEF469
:10936A00E8EBFC203300CFF0EEF4E8EBFC2032000F
:10937A00CFF0EEF4E8EBFC203100CFF0EEF4E8EBAE
:10938A00FC203000536E416700536E506200CFF0EC
:10939A00E8EDFFF2EE202000C2DBC1D0C0D2DC0033
:1093AA00C2DBCACB00C2CACB00CDE0F1F2F0EEE8D4
:1093BA00F2FC00C7E2F3EAEEE2FBE520F1E8E3EDB6
:1093CA00E0EBFB00CFF0E5E4F3F1F2E0EDEEE2EAE8
:1093DA00E800D3ECEEEBF7E0EDE8FF00C2F0E5ECD5
:1093EA00FF20EFE0E9EAE80020C4E0F2F7E8EA202B
:1093FA00EDE8E62E20EDE0E3F0E5E2E0F2E5EBFF52
:10940A000020C4E0F2F7E8EA20ECE5F1F2E020EF10
:06941A00E0E9EAE80000B1
:00000001FF
